:0200000480007A
:10000000B72F0000938F0F8073900F3015A8130047
:100010000000130000001300000013000000130094
:100020000000130000001300000013000000130084
:100030000000130000001300000013000000010086
:10004000970200009382020C73905230814001416C
:100050008141014281420143814301448144014580
:100060008145014681460147814701488148014950
:100070008149014A814A014B814B014C814C014D20
:10008000814D014E814E014F814F971102009381A6
:1000900021C3170502001305E546979503009385D4
:1000A000A57201461122170502001305A540970508
:1000B00002009385A5400146C52817A50300130536
:1000C000E57097B503009385257037B6ABAB130683
:1000D000B6BAD92817B103001301416FEF40807DF4
:1000E000860293D21200F512638802008242110147
:1000F0006F00001073002030824211017300203025
:10010000711116C0F3222034E3CC02FC82421101AB
:10011000130141F806C20AC40EC612C816CA1ACC88
:100120001ECE22D026D22AD42ED632D836DA3ADCC7
:100130003EDEC2C0C6C2CAC4CEC6D2C8D6CADACC97
:10014000DECEE2D0E6D2EAD4EED6F2D8F6DAFADCA7
:10015000FEDE73252034F32510340A8601A07310C7
:10016000153492402241B2414242D2426243F243AC
:10017000025492542255B2554256D2566257F25703
:10018000064896482649B649464AD64A664BF64B33
:10019000065C965C265DB65D465ED65E665FF65F83
:1001A0001301C1077300203010C16374B50011053D
:1001B000E5BF828000000000000000000000000099
:1001C000000000000000000000000000000000002F
:1001D000000000000000000000000000000000001F
:1001E000000000000000000000000000000000000F
:1001F000197106C00AC20EC412C616C81ACA1ECC8D
:1002000022CE26D02AD22ED432D636D83ADA3EDCC6
:1002100042DEC6C0CAC2CEC4D2C6D6C8DACADECC96
:10022000E2CEE6D0EAD2EED4F2D6F6D8FADAFEDCA6
:100230009702020083A2022823A02200F322103496
:1002400096DEEF006030170102000321A126024173
:10025000F65273901234B72200009382028873A082
:10026000023082403242C2425243E24372448254DC
:100270001255A2553256C2565257E2577258864806
:100280001649A649364AC64A564BE64B764C865C1A
:10029000165DA65D365EC65E565FE65F0961730059
:1002A0002030970202009382E22523A0120023A2AD
:1002B000220023A4320023A6420023A8520023AA2E
:1002C000620023AC720023AE820023A0920223A21C
:1002D000A20223A4B20223A6C20223A8D20223AA06
:1002E000E20223ACF20223AE020323A0120523A2F2
:1002F000220523A4320523A6420523A8520523AADA
:10030000620523AC720523AE820523A0920723A2C7
:10031000A20723A4B20723A6C20723A8D20723AAB1
:10032000E20723ACF207EF40804D170102000321E2
:1003300061180241F65273901234B7220000938282
:10034000028873A0023082403242C2425243E243EA
:10035000724482541255A2553256C2565257E25731
:10036000725886481649A649364AC64A564BE64B45
:10037000764C865C165DA65D365EC65E565FE65FB1
:10038000096173002030970202009382A21783A0B4
:10039000020003A1420083A1820003A2C20083A243
:1003A000020103A3420183A3820103A4C20183A427
:1003B000020203A5420283A5820203A6C20283A60B
:1003C000020303A7420383A7820303A8C20383A8EF
:1003D000020403A9420483A9820403AAC20483AAD3
:1003E000020503AB420583AB820503ACC20583ACB7
:1003F000020603AD420683AD820603AEC20683AE9B
:10040000020703AFC20983AF820782807370043092
:10041000197106C00AC20EC412C616C81ACA1ECC6A
:1004200022CE26D02AD22ED432D636D83ADA3EDCA4
:1004300042DEC6C0CAC2CEC4D2C6D6C8DACADECC74
:10044000E2CEE6D0EAD2EED4F2D6F6D8FADAFEDC84
:100450009702020083A2020623A0220086DEEF108C
:10046000B040170102000321E1040241F6527390EB
:100470001234B72200009382028873A002308240B7
:100480003242C2425243E243724482541255A25550
:100490003256C2565257E257725886481649A649F4
:1004A000364AC64A564BE64B764C865C165DA65DD0
:1004B000365EC65E565FE65F0961730020309707BF
:1004C00002009387E7FF9843FD576305F7007370B9
:1004D000043001A07370043001A041112AC6B24754
:1004E000739047300100410182804111F327403071
:1004F0003EC673F04330B2473E85410182804111D0
:100500002AC62EC432C2B247F1173EC62247B247AE
:1005100098C3B247938787FA3EC61247B24798C33B
:10052000B247A1173EC68E873E87B24798C3B247EF
:10053000D1173EC6170700001307A7F8B24798C3A4
:10054000B2473E8541018280411106C6EF40A0239B
:10055000EF10D014AA8799C3EF1010310100B240F8
:100560004101828041112AC6B24713878700B247F2
:10057000D8C3B2477D5798C7B24713878700B247A1
:10058000D8C7B24713878700B24798CBB24723A09A
:10059000070001004101828041112AC6B24723A809
:1005A000070001004101828001112AC62EC4B24712
:1005B000DC433ECEA2477247D8C3F2479847A247D2
:1005C00098C7F2479C472247D8C3F247224798C7AB
:1005D000A247324798CBB2479C4313871700B247D4
:1005E00098C301000561828001112AC62EC4A2476A
:1005F0009C433ECC6247FD576316F700B2479C4BC5
:100600003ECE31A8B247A1073ECE21A0F247DC433F
:100610003ECEF247DC439C436247E379F7FEF24764
:10062000D843A247D8C3A247DC43224798C7A24772
:10063000724798C7F2472247D8C3A247324798CBA0
:10064000B2479C4313871700B24798C30100056166
:10065000828001112AC6B2479C4B3ECEB247DC4392
:100660003247184798C7B2479C4732475843D8C3C8
:10067000F247DC4332476316F700B2479847F24728
:10068000D8C3B24723A80700F2479C431387F7FF5C
:10069000F24798C3F2479C433E8505618280797199
:1006A00006D622D42AC62EC4B2473ECEF24781E7F0
:1006B0007370043001A0EF202057F2478043F247C7
:1006C000D85FF247BC43BE853A85EF70A066AA8723
:1006D0003307F400F247D8C3F24723AC0702F247CE
:1006E0009843F24798C7F2478043F247DC5F13878D
:1006F000F7FFF247BC43BE853A85EF70A063AA8737
:100700003307F400F247D8C7F2477D57F8C3F247E2
:100710007D57B8C7A24799EFF2479C4B8DC7F24768
:10072000C1073E85EF1090402A878547631DF7007B
:10073000F13911A8F247C1073E852D35F24793875D
:1007400047023E850535EF20005185473E85B25072
:10075000225445618280797106D62AC62EC4B2879A
:10076000A303F10002CCB24781E77370043001A00B
:10077000A24799E302CE01A8A2453245EF70805B03
:10078000AA8785073ECEF247938747053E85EF301F
:10079000805C2ACAD24785CFA24789E7D247524711
:1007A00098C331A0D24713874705D24798C3D24791
:1007B0003247D8DFD2472247B8C385455245C535B1
:1007C000D247034771002388E704D2473ECCE24773
:1007D00081E77370043001A0E2473E85B250456165
:1007E0008280797106D6AA87A307F1001305400518
:1007F000EF3060562ACEF247B9CFF24723A2070066
:10080000F24723A00700F24723A40700F24723A6DC
:100810000700F24723AC0702F2470547D8DFF2474B
:1008200023A00704F2477D57F8C3F2477D57B8C7A6
:10083000F2470347F1002388E704F247C1073E85EA
:100840001533F247938747023E85293B814601468F
:10085000814572453122F2473E85B2504561828022
:10086000797106D622D42AC6B2473ECCE24781E748
:100870007370043001A0E247C043EF20001DAA8737
:100880006313F402E247DC471387F7FFE247D8C758
:10089000E247DC4791E78146014681456245C92030
:1008A00085473ECE11A002CEF2473E85B25022547B
:1008B00045618280797106D622D42AC62EC4B247F9
:1008C0003ECCE24781E77370043001A0E247C043A9
:1008D000EF20A017AA87631BF400E247DC471387C9
:1008E0001700E247D8C785473ECE0DA08146224675
:1008F00081456245252E2ACE724785476318F70049
:10090000E247DC4713871700E247D8C7F2473E8526
:10091000B250225445618280797106D62AC62EC40F
:10092000B24781E77370043001A02247B24763F5F4
:10093000E7007370043001A0094681453245213D2E
:100940002ACEF24781C7F247224798DFF24781E774
:100950007370043001A0F2473E85B2504561828039
:10096000397106DE2AC62EC432C236C002D6B2475C
:100970003ED4A25781E77370043001A0A24781E7FB
:10098000A257BC4399E3854711A0814781E7737063
:10099000043001A0024789476317F700A257D85FC8
:1009A00085476314F700854711A0814781E773707D
:1009B000043001A0EF20C00AAA8799E3924799E387
:1009C000854711A0814781E77370043001A0EF20B3
:1009D000A025A257985FA257DC5F6366F700024725
:1009E0008947631DF7020246A245225565232AD294
:1009F000A257DC5389CFA257938747023E85EF1059
:100A0000F0122A8785476317F700093421A092570F
:100A100091C3ED3AEF202024854771A8924789E7DA
:100A2000EF206023814741A8B25799E77C083E85B3
:100A3000EF10702785473ED6EF20E021EF10401AD7
:100A4000EF20801EA257F843FD576315F700A25709
:100A500023A20704A257B847FD576315F700A25712
:100A600023A40704EF20201F58007C08BA853E8588
:100A7000EF107026AA879DEB2255EF006071AA87C0
:100A80008DC3A257C1071247BA853E85EF10E070AB
:100A900022551525EF108016AA87E39A07F2BD327A
:100AA0003DB72255092DEF10601515B722552125A8
:100AB000EF10C01481473E85F25021618280797128
:100AC00006D62AC62EC432C236C0B2473ECCE24752
:100AD00081E77370043001A0A24781E7E247BC437D
:100AE00099E3854711A0814781E77370043001A025
:100AF000024789476317F700E247D85F85476314C9
:100B0000F700854711A0814781E77370043001A089
:100B1000E93AAA873ECAE247985FE247DC5F63662C
:100B2000F700024789476315F7040246A24562456C
:100B30009521E247B847FD576313F702E247DC53BC
:100B40008DC7E247938747023E85EF10207EAA8734
:100B500089CF924799CB9247054798C339A0E2477E
:100B6000BC4713871700E247B8C785473ECE11A0A0
:100B700002CED2473E859532F2473E85B25045615E
:100B80008280797106D62AC62EC4B2473ECCE2478F
:100B900081E77370043001A0E247BC4381C77370E2
:100BA000043001A0E2479C4381E7E247DC4399E33C
:100BB000854711A0814781E77370043001A0353269
:100BC000AA873ECAE247985FE247DC5F6377F70493
:100BD000E2479C5F13871700E24798DFE247B84778
:100BE000FD576313F702E247DC538DC7E247938753
:100BF00047023E85EF108073AA8789CFA24799CB21
:100C0000A247054798C339A0E247BC47138717009E
:100C1000E247B8C785473ECE11A002CED2473E85F7
:100C20006D38F2473E85B25045618280397106DEEB
:100C30002AC62EC432C236C002D6B2473ED4A2570C
:100C400081E77370043001A0A24781E7A257BC433B
:100C500099E3854711A0814781E77370043001A0B3
:100C6000EF101060AA8799E3924799E3854711A096
:100C7000814781E77370043001A0EF10F07AA2572A
:100C80009C5FB5CBA257DC473ED2A2452255F92E38
:100C9000824795EFA2579C5F1387F7FFA25798DF13
:100CA000A2579C4391E7EF2060022A87A257D8C33E
:100CB000A2579C4B8DCFA257C1073E85EF1000670E
:100CC0002A8785476315F702EFF04FF40DA0A2576E
:100CD0001257D8C7A257DC5399CBA2579387470224
:100CE0003E85EF10A064AA8799C3EFF02FF2EF10B2
:100CF000907685475DA8924789E7EF10D0758147C8
:100D00006DA0B25799E77C083E85EF10C079854702
:100D10003ED6EF105074EF00B06CEF10F070A25799
:100D2000F843FD576315F700A25723A20704A25703
:100D3000B847FD576315F700A25723A40704EF1027
:100D4000907158007C08BA853E85EF10C078AA875C
:100D5000A1EB2255CD2EAA879DCFA2579C4391EBA4
:100D6000EF10906CA257DC433E85EF107052EF10ED
:100D7000906EA257938747021247BA853E85EF10BF
:100D8000C04122550D2EEF007067AA87E39707EE4A
:100D9000EFF0CFE7DDB52255392EEF003066F1BD1B
:100DA0002255112EEF00906581473E85F25021615A
:100DB0008280797106D62AC62EC432C2B2473ECC92
:100DC000E24781E77370043001A0A24781E7E24760
:100DD000BC4399E3854711A0814781E773700430D4
:100DE00001A0EFF08FF0AA873ECAE2479C5FA1CB3B
:100DF000A2456245A52CE2479C5F1387F7FFE247B7
:100E000098DFE247F843FD576312F702E2479C4B35
:100E100085C7E247C1073E85EF104051AA8789CFB9
:100E2000924799CB9247054798C339A0E247FC43C4
:100E300013871700E247F8C385473ECE11A002CEC4
:100E4000D2473E85EFF06FE9F2473E85B2504561EB
:100E50008280797106D62AC62EC4B2473ECCE247BC
:100E600081E77370043001A0A24781E7E247BC43E9
:100E700099E3854711A0814781E77370043001A091
:100E8000E247BC4381E77370043001A0EFF0EFE567
:100E9000AA873ECAE2479C5F89CFE247DC473EC84B
:100EA000A2456245E122E2474247D8C785473ECE88
:100EB00011A002CED2473E85EFF02FE2F2473E85E9
:100EC000B25045618280797106D62AC6B24781E761
:100ED0007370043001A0EF103055B2479C5F3ECED6
:100EE000EF107057F2473E85B250456182807971AC
:100EF00006D62AC6B2473ECEF24781E77370043069
:100F000001A0EF107052F247D85FF2479C5FB30721
:100F1000F7403ECCEF103054E2473E85B250456179
:100F2000828001112AC6B24781E77370043001A0A4
:100F3000B2479C5F3ECEF2473E8505618280797163
:100F400006D62AC6B2473ECEF24781E77370043018
:100F500001A07245E5247245EF20F0720100B25005
:100F60004561828041112AC6B247FC473E85410156
:100F7000828041112AC62EC4B2472247F8C7010019
:100F80004101828041112AC6B24783C707053E85C9
:100F900041018280797106D62AC62EC432C202CEA1
:100FA000B247BC4391EFB2479C43D5E7B247DC431D
:100FB0003E85EF10903B2ACEB24723A2070061A8DE
:100FC000924785EFB2479847B247BC433E86A24559
:100FD0003A85EF20F079B2479847B247BC433E9735
:100FE000B24798C7B2479847B247DC436365F706F4
:100FF000B2479843B24798C7B9A8B247D847B24753
:10100000BC433E86A2453A85EF209076B247D8474A
:10101000B247BC43B307F0403E97B247D8C7B24788
:10102000D847B2479C43637BF700B247D843B247E7
:10103000BC43B307F0403E97B247D8C71247894731
:10104000631BF700B2479C5F99C7B2479C5F138749
:10105000F7FFB24798DFB2479C5F13871700B2478C
:1010600098DFF2473E85B25045618280011106CE7D
:101070002AC62EC4B247BC439DCBB247D847B2471D
:10108000BC433E97B247D8C7B247D847B247DC43C4
:101090006366F700B2479843B247D8C7B247D8470C
:1010A000B247BC433E86BA852245EF20706C0100F2
:1010B000F24005618280011106CE2AC6EF10D036BB
:1010C00025A0B247DC5395C7B247938747023E85B8
:1010D000EF10C025AA8799C3EF104049B247BC471B
:1010E0001387F7FFB247B8C7B247BC47E34BF0FCE2
:1010F00011A00100B2477D57B8C7EF10D035EF10EF
:10110000B0321DA0B2479C4B8DC7B247C1073E8588
:10111000EF10C021AA8799C3EF104045B247FC43A6
:101120001387F7FFB247F8C3B247FC43E34CF0FC28
:1011300011A00100B2477D57F8C3EF10D031010074
:10114000F24005618280797106D62AC6EF10D02D53
:10115000B2479C5F81E785473ECE11A002CEEF10DB
:10116000902FF2473E85B2504561828001112AC618
:10117000B24781E77370043001A0B2479C5F81E7FA
:1011800085473ECE11A002CEF2473E8505618280A2
:10119000797106D62AC6EF103029B247985FB24758
:1011A000DC5F6315F70085473ECE11A002CEEF103D
:1011B000902AF2473E85B2504561828001112AC6CD
:1011C000B24781E77370043001A0B247985FB2471D
:1011D000DC5F6315F70085473ECE11A002CEF247D3
:1011E0003E850561828001112AC62EC402CE81A0EF
:1011F0001787030013078759F2478E07BA979C4356
:1012000085E71787030013076758F2478E07BA97D9
:10121000224798C31787030013074757F2478E07E3
:10122000BA973247D8C301A8F24785073ECE724726
:101230009D47E3FFE7FA01000561828001112AC69C
:1012400002CE0DA81787030013074754F2478E07F5
:10125000BA97DC433247631CF70017870300130774
:10126000E752F2478E07BA9723A0070001A8F2477A
:1012700085073ECE72479D47E3F6E7FC0100056116
:101280008280797106D62AC62EC432C2B2473ECEBB
:10129000EF109019F247F843FD576315F700F24736
:1012A00023A20704F247B847FD576315F700F2473A
:1012B00023A40704EF10301AF2479C5F89EBF24732
:1012C000938747021246A2453E85EF00907E724505
:1012D000DD330100B25045618280397106DE2ACECD
:1012E0002ECC36C83AC63EC442C246C0B287231B83
:1012F000F100F24781E77370043001A03247914753
:1013000063F5E7007370043001A0835761019245D3
:101310003E85EF1080512AD4A257638F0712A2573F
:10132000985B83566101B7070040FD17B6978A079F
:10133000BA973ED29257F19B3ED292578D8B81C77E
:101340007370043001A0835761013E8782463246A4
:10135000E2452255EF10E0274246F2451255EFF0E4
:101360000F9A2A87A25798C3A24781C7A24722573C
:1013700098C3EF10700B97F701009387A72D9C433C
:101380001387170097F701009387C72C98C397F727
:101390000100938727129C4395E397F701009387F9
:1013A0006711225798C397F701009387A72A98439C
:1013B0008547631AF702EF10C02C35A097F701009C
:1013C0009387072A9C4385E397F701009387870E4D
:1013D0009C43DC5732476368F70097F70100938717
:1013E000670D225798C397F70100938767289C439E
:1013F0001387170097F701009387872798C397F7FC
:1014000001009387E7269843A257B8C7A257D85739
:1014100097F70100938787249C4363F9E700A2575D
:10142000D85797F701009387672398C3A257D857D7
:10143000BA878A07BA978A0717F701001307471474
:101440003E97A2579107BE853A85EFF0EF95854705
:101450003ED6EF10500019A0FD573ED632578547B3
:101460006313F70297F701009387871F9C4381CF8F
:1014700097F70100938707049C43DC57324763F4D6
:10148000E700EFE0BFF8B2573E85F250216182805D
:10149000797106D62AC6EF102079B24799E797F7F7
:1014A0000100938727019C4311A0B2473ECEF2472B
:1014B00091073E85EFF0EF99F2479C5791C7F247AD
:1014C000E1073E85EFF0EF98F2479107BE8517F5EB
:1014D000010013056515EFF02F8D97F70100938735
:1014E000E7159C431387170097F7010093870715AB
:1014F00098C397F701009387A7179C43138717009A
:1015000097F701009387C71698C3EF10C07497F739
:1015100001009387E7149C439DCB97F701009387C5
:1015200067F99C437247631EF70097F701009387A2
:10153000A7149C4381C77370043001A0EFE01FED36
:1015400039A0EF10606EEF10A04BEF10C0700100DB
:10155000B25045618280797106D62AC62EC402CE69
:10156000B24781E77370043001A0A24781E773702E
:10157000043001A097F70100938707109C4381C7AF
:101580007370043001A0A92D97F701009387C70C51
:101590009C433ECCB2479C432247BA973ECAB247CF
:1015A0009C436247637EF700B2479C435247637493
:1015B000F7025247E24763F0E70285473ECE21A893
:1015C000B2479C4352476366F7005247E24763F4D1
:1015D000E70085473ECEB247524798C3F24789CFCE
:1015E00097F70100938707ED9C4391073E85EFF045
:1015F0004F865245EF10001B11252AC8C24799E3B8
:10160000EFE0DFE00100B25045618280797106D6DB
:101610002AC602CEB247A9C397F701009387C70530
:101620009C4381C77370043001A05D2B97F70100C4
:10163000938787029C433247BA973ECC97F70100C5
:10164000938747E79C4391073E85EFF08F80624583
:10165000EF10401565232ACEF24799E3EFE01FDB38
:101660000100B25045618280797106D62AC6B24720
:101670003ECCE24781E77370043001A097F7010088
:10168000938747E39C4362476314F70002CEBDA0F3
:10169000EF108059E247DC4B3ECAEF10C05B97F772
:1016A00001009387A7F69C435247630AF70097F718
:1016B00001009387E7F59C4352476315F70089477C
:1016C0003ECE2DA8524797F70100938767F7631B1B
:1016D000F700E2479C5781E78D473ECE05A089473A
:1016E0003ECE29A8524797F701009387E7F3631589
:1016F000F70091473ECE19A085473ECEF2473E8582
:10170000B25045618280797106D62AC6EF10C05169
:10171000B24799E797F701009387C7D99C4311A077
:10172000B2473ECEF247DC573ECCEF10C052E24704
:101730003E85B25045618280797106D62AC6EFE0B7
:10174000DFDAAA873ECEB24799E797F70100938781
:1017500067D69C4311A0B2473ECCE247DC573ECA55
:10176000F2473E85EFE07FD7D2473E85B2504561D4
:101770008280797106D62AC62EC402CE22479147AE
:1017800063F5E7007370043001A02247914763F4CA
:10179000E70091473EC4EF102049B24799E797F719
:1017A0000100938727D19C4311A0B2473ECCE2476A
:1017B000BC4B3ECA5247A247630AF70E2247D247A4
:1017C00063F6E70297F701009387C7CE9C43624711
:1017D0006308F70297F701009387C7CD9C43DC5756
:1017E0002247636FF70085473ECE19A897F701009F
:1017F000938747CC9C4362476314F70085473ECEEE
:10180000E247DC573EC8E247B84BE247DC57631576
:10181000F700E2472247D8D7E2472247B8CBE24752
:101820009C4F63C707001547A2471D8FE24798CF1B
:10183000E247D44B4247BA878A07BA978A0717F715
:1018400001001307E7D3BA976394F600854711A008
:101850008147B9C7E24791073E85EFE09FDFE24746
:10186000D85797F70100938767DF9C4363F9E70038
:10187000E247D85797F70100938747DE98C3E247BE
:10188000D857BA878A07BA978A0717F7010013074C
:1018900027CF3E97E2479107BE853A85EFE0DFD03C
:1018A000724785476314F700EFE05FB6EF10A03A88
:1018B0000100B25045618280797106D62AC6EF10C8
:1018C000A036B24799E797F701009387A7BE9C43DC
:1018D00011A0B2473ECEF24791073E85EFE07FD799
:1018E000F2479C5791C7F247E1073E85EFE07FD66C
:1018F000F2479107BE8517F50100130565D4EFE0A7
:10190000BFCAEF10403597F701009387A7BA9C43F1
:1019100072476319F70497F70100938767D49C43D4
:1019200089CF97F70100938727D59C4381C77370B0
:10193000043001A0EFE09FAD91A097F701009387DD
:1019400027D0984397F701009387C7D09C4363192A
:10195000F70097F701009387E7B523A0070039A8A0
:10196000212729A897F70100938787CF9C4399C720
:10197000EF10802BEF10C008EF10E02D0100B250E7
:101980004561828001112AC602CEB2473ECCB247E1
:1019900081E77370043001A0E247D84B97F701004C
:1019A000938707CA6314F700854711A0814795C341
:1019B000E247985797F701009387C7C5630BF70075
:1019C000E2479C5799E3854711A0814799C3854712
:1019D0003ECEF2473E8505618280797106D62AC6E1
:1019E000B2473ECEB24781E77370043001A0F247A0
:1019F000C9C797F701009387E7AB9C437247630E13
:101A0000F706EF1060227245B53F2A8785476314B9
:101A1000F706F24791073E85EFE0BFC3F247D8577C
:101A200097F70100938787C39C4363F9E700F24768
:101A3000D85797F70100938767C298C3F247D857E2
:101A4000BA878A07BA978A0717F70100130747B3BF
:101A50003E97F2479107BE853A85EFE0FFB4F24723
:101A6000D85797F701009387E7A49C43DC5763643A
:101A7000F700EFE0BF99EF10001E0100B250456182
:101A80008280797106D62AC602CEB2473ECCB247D2
:101A900081E77370043001A0EFE03FA5AA873ECA3A
:101AA0006245CD352A8785476314F70897F701000B
:101AB000938787BC9C43A5E7E247D85797F7010077
:101AC0009387479F9C43DC576364F70085473ECE6E
:101AD000E24791073E85EFE0DFB7E247D85797F737
:101AE00001009387A7B79C4363F9E700E247D85703
:101AF00097F70100938787B698C3E247D857BA870C
:101B00008A07BA978A0717F70100130767A73E9756
:101B1000E2479107BE853A85EFE01FA911A8E24789
:101B2000E107BE8517F501001305C5AEEFE0DFA79D
:101B3000D2473E85EFE07F9AF2473E85B25045613D
:101B40008280011106CE81480148814701478146C4
:101B50001306004097E501009385C54A171500005C
:101B6000130585A5EFF06FF72AC632478547631541
:101B7000F700EF10C06D2AC6324785476319F70298
:101B80007370043097F701009387C7AE7D5798C3F1
:101B900097F701009387C7AC054798C397F70100F3
:101BA000938787AB23A00700EFE0AFEF31A0B247E8
:101BB00081E77370043001A00100F240056182806A
:101BC000411106C67370043097F70100938747A947
:101BD00023A00700EFE02FFB0100B240410182800B
:101BE00097F70100938747A99C431387170097F73E
:101BF0000100938767A898C301008280011106CE77
:101C000002C697F70100938727A79C4381E773706B
:101C1000043001A0EF10400197F701009387C7A59A
:101C20009C431387F7FF97F701009387E7A498C3B6
:101C300097F70100938747A49C436390071097F799
:101C40000100938727A19C436389070E59A097F74A
:101C500001009387279CDC47DC473EC4A247E1078D
:101C60003E85EFE01F9FA24791073E85EFE07F9EF4
:101C7000A247D85797F701009387479E9C4363F983
:101C8000E700A247D85797F701009387279D98C38D
:101C9000A247D857BA878A07BA978A0717F7010069
:101CA0001307078E3E97A2479107BE853A85EFE05E
:101CB000BF8FA247D85797E701009387A77F9C4320
:101CC000DC576368F70097F701009387E7990547AA
:101CD00098C397F701009387E7939C43ADFB97F771
:101CE0000100938727989C438DCF35A0452AAA876A
:101CF00099C797F7010093872797054798C397F7E8
:101D00000100938727969C431387F7FF97F70100FD
:101D10009387479598C397F701009387A7949C43AF
:101D2000F1F797F701009387279498438547631647
:101D3000F70085473EC6EFE06FEDEF00D071B24788
:101D40003E85F24005618280011106CEEF00D06D24
:101D500097F70100938747909C433EC6EF00B06F12
:101D6000B2473E85F24005618280011106CEEFE068
:101D7000CFF7AA873EC697F701009387E78D9C436C
:101D80003EC4B2473E85EFE04FF5A2473E85F240A4
:101D90000561828097F701009387C78B9C433E853E
:101DA0008280797106D62AC62EC432C202CE9547E9
:101DB0003ECC3D3597F701009387C7899C43224766
:101DC0006368F70CE247FD173ECCF24796073247AF
:101DD000B306F7006247BA878A07BA978A0717E7F8
:101DE00001001307E779BA970546BE853685EF00EF
:101DF000902A2A87F247BA973ECEE247E1F7F247A8
:101E0000960732473E9797F70100938727809C43B8
:101E10000946BE853A85EF0010282A87F247BA970F
:101E20003ECEF247960732473E9797E701009387E9
:101E3000277E9C430946BE853A85EF00D0252A8738
:101E4000F247BA973ECEF24796073247BA97114605
:101E500097E501009385457D3E85EF00D0232A87D5
:101E6000F247BA973ECEF24796073247BA970D46E9
:101E700097E501009385C57C3E85EF00D0212A8738
:101E8000F247BA973ECE924781C7924723A00700F8
:101E9000B533F2473E85B25045618280797106D6EE
:101EA00002CE97E701009387277D9C43639507182F
:101EB00097E701009387477A9C431387170097E7BA
:101EC00001009387677998C397E701009387C778E4
:101ED0009C433ECCE247B9EF97E701009387077335
:101EE0009C439C4381C77370043001A097E70100B5
:101EF0009387C7719C433ECA97E701009387477158
:101F0000984397E701009387677098C397E70100AC
:101F100093870770524798C397E701009387077527
:101F20009C431387170097E701009387277498C392
:101F3000EF00102D97E701009387C7739C4362471A
:101F40006365F70C97E701009387476C9C439C43BC
:101F500099E3854711A0814781CB97E701009387DB
:101F600067717D5798C355A097E701009387076A6B
:101F70009C43DC47DC473EC8C247DC433EC6624761
:101F8000B2476379F70097E701009387A76E32475E
:101F900098C3A5A8C24791073E85EFE08FEBC247E3
:101FA0009C5791C7C247E1073E85EFE08FEAC247E1
:101FB000D85797E701009387676A9C4363F9E70066
:101FC000C247D85797E701009387476998C3C2472C
:101FD000D857BA878A07BA978A0717E70100130705
:101FE000275A3E97C2479107BE853A85EFE0CFDB7F
:101FF000C247D85797E701009387C74B9C43DC57EC
:10200000E362F7F485473ECE35BF97E7010093873B
:10201000674A9C43D85797E6010093866656BA876D
:102020008A07BA978A07B6979843854763F1E7020C
:1020300085473ECE29A897E701009387A7629C4376
:102040001387170097E701009387C76198C397E745
:102050000100938767619C4399C385473ECEF24751
:102060003E85B25045618280011106CE97E701009E
:10207000938787609C4381CB97E701009387C75E76
:10208000054798C339A297E701009387E75D23A02E
:10209000070097E701009387E7419C439C5B3EC69E
:1020A000B7A7A5A59387575A3EC4B2479C4322477A
:1020B0006314F702B24791079C432247631EF7005F
:1020C000B247A1079C4322476318F700B247B10704
:1020D0009C4322476308F70497E701009387873DF5
:1020E000984397E701009387E73C9C439387470316
:1020F000BE853A85EF20F00A35A097E70100938767
:10210000E7559C4381E77370043001A097E7010015
:102110009387C7549C431387F7FF97E70100938782
:10212000E75398C397E7010093874753984397E68F
:1021300001009386E644BA878A07BA978A07B6975A
:102140009C43C5DF97E70100938747519843BA87BF
:102150008A07BA978A0717E7010013076742BA97F9
:102160003EC29247DC43D8439247D8C39247D843F4
:102170009247A1076317F7009247DC43D843924781
:10218000D8C39247DC43D84797E70100938787324B
:1021900098C30100F24005618280797106D62AC693
:1021A0002EC4B24781E77370043001A097E70100A5
:1021B000938747309C43E107BE853245EFE0CFC2AD
:1021C00097E701009387072F9C4391073E85EFE037
:1021D0004FC82247FD576310F70297E70100938726
:1021E000672D9C439107BE8517E501001305454502
:1021F000EFE08FBB19A897E701009387E7459C4361
:102200002247BA973ECE7245712B0100B25045610C
:102210008280797106D62AC62EC432C2B24781E7BF
:102220007370043001A097E701009387E7449C4353
:1022300081E77370043001A097E701009387872737
:102240009C43A24637070080558F98CF97E701003F
:10225000938747269C43E107BE853245EFE0CFB424
:1022600097E70100938707259C4391073E85EFE0A0
:102270004FBE1247FD576310F70297E7010093879F
:1022800067239C439107BE8517E501001305453B75
:10229000EFE08FB119A897E701009387E73B9C43D4
:1022A0001247BA973ECE7245F5290100B2504561FA
:1022B0008280797106D62AC62EC432C2B24781E71F
:1022C0007370043001A097E701009387A71E9C4319
:1022D000E107BE853245EFE02FAD97E70100938718
:1022E000671D9C4391073E85EFE0AFB612478547D7
:1022F0006310F70297E701009387C71B9C43910780
:10230000BE8517E501001305A533EFE0EFA919A875
:1023100097E70100938747349C432247BA973ECE04
:10232000724549210100B25045618280797106D61B
:102330002AC6B247DC47DC473ECCE24781E77370F0
:10234000043001A0E247E1073E85EFE08FB097E758
:102350000100938767329C43A1EBE24791073E85DA
:10236000EFE02FAFE247D85797E701009387072F99
:102370009C4363F9E700E247D85797E7010093874A
:10238000E72D98C3E247D857BA878A07BA978A07D2
:1023900017E701001307C71E3E97E2479107BE8566
:1023A0003A85EFE06FA011A8E247E107BE8517E587
:1023B000010013052526EFE02F9FE247D85797E746
:1023C00001009387270F9C43DC5763FBE700854799
:1023D0003ECE97E7010093872729054798C311A0B0
:1023E00002CEF2473E85B25045618280797106D6B1
:1023F0002AC62EC497E70100938707289C4381E7EC
:102400007370043001A02247B70700805D8FB24788
:1024100098C3B247DC473ECCE24781E77370043093
:1024200001A03245EFE0EFA2E24791073E85EFE0E1
:102430004FA2E247D85797E70100938727229C4392
:1024400063F9E700E247D85797E701009387072130
:1024500098C3E247D857BA878A07BA978A0717E717
:1024600001001307E7113E97E2479107BE853A85C1
:10247000EFE08F93E247D85797E7010093878703F0
:102480009C43DC5763FBE70085473ECE97E701009E
:102490009387871D054798C311A002CEF2473E855A
:1024A000B2504561828041112AC6B24781E77370FC
:1024B000043001A097E701009387471B9843B24778
:1024C00098C397E70100938727199843B247D8C369
:1024D000010041018280797106D62AC62EC4B24716
:1024E00081E77370043001A0A24781E77370043064
:1024F00001A01D2F97E70100938707169C433ECC50
:10250000A2479843FD576314F70002CE91A8B24743
:10251000984397E70100938767159C43630AF70088
:10252000B247DC4362476365F70085473ECE0DA89E
:10253000B247DC4362471D8FA2479C436370F7029A
:10254000A2479843B247D443E247B387F6403E9749
:10255000A24798C33245813F02CE19A085473ECE9F
:10256000DD2DF2473E85B2504561828097E701003C
:102570009387870F054798C30100828001112AC6FF
:10258000B24799C7B2473ECCE247FC473ECE11A0C6
:1025900002CEF2473E850561828001112AC62EC413
:1025A000B24791C7B2473ECEF2472247F8C7010073
:1025B00005618280011106CE2AC6852297E70100B7
:1025C000938707FC98438547E3F9E7FEEFD01FE4C4
:1025D000EDB7397106DE2ACE2ECC32CA36C8BA879C
:1025E0002317F10002D625A06247B257BA9703C756
:1025F0000700F246B257B697238AE7026247B257FE
:10260000BA9783C7070089CBB25785073ED63257A2
:10261000BD47E3FBE7FC11A00100F247A3810704DB
:102620005247914763F4E70091473ECAF247524749
:10263000D8D7F2475247B8CBF24723AA0704F2474C
:1026400091073E85EFD05FF5F247E1073E85EFD079
:10265000BFF4F247724798CB1547D2471D8FF24718
:1026600098CFF2477247D8D3F24723A20704F24724
:1026700023AC0704F24723AE07040100F2502161A6
:102680008280011106CE02C60DA03247BA878A07A2
:10269000BA978A0717E70100130787EEBA973E85B6
:1026A000EFD05FECB24785073EC632479147E3FE65
:1026B000E7FC17E501001305E5F2EFD0BFEA17E5E7
:1026C0000100130565F3EFD0FFE917E501001305DD
:1026D00065F4EFD03FE917E501001305E5F4EFD00D
:1026E0007FE817E501001305A5F5EFD0BFE797E7F1
:1026F00001009387A7F117E701001307A7EE98C31E
:1027000097E701009387C7F017E701001307C7EEAB
:1027100098C30100F24005618280011106CE8DA8A8
:10272000EFF00FCC97E70100938707F09C4393B736
:10273000170093F7F70F3EC6EFF04FCCB247A9EB67
:10274000E52197E70100938727EEDC47DC473EC48D
:10275000A24791073E85EFD0DFEF97E7010093870F
:1027600067EF9C431387F7FF97E70100938787EE96
:1027700098C397E70100938767EC9C431387F7FFA3
:1027800097E70100938787EB98C3F1212245912CAD
:1027900097E70100938787EA9C43D9F30100F24051
:1027A00005618280011106CE2AC697E70100938752
:1027B00067D09C433247D8C397E701009387C7E9A6
:1027C0009C4332476372F70297E70100938747E41F
:1027D000984397E701009387E7CD9C439107BE8517
:1027E0003A85EFD07FE035A897E70100938707E2AD
:1027F000984397E701009387E7CB9C439107BE85F9
:102800003A85EFD07FDE97E701009387A7E69C43E8
:1028100032476378F70097E701009387A7E53247CF
:1028200098C30100F24005618280797106D6AA87BB
:102830002EC42317F100A24789EB8357E1008A07D2
:102840003E85EF104051AA8711A0A2473ECCE24737
:1028500085C313050006EF1000502ACEF24789C742
:10286000F247624798DB31A06245EF10C06111A0CA
:1028700002CEF24781CFF247985B8357E1008A0787
:102880003E869305500A3A85EF104075F2473E8523
:10289000B25045618280397106DE22DC2AC62EC420
:1028A00032C202D6A2479C43638D070EA2473ED494
:1028B000A257DC43D843A257D8C3A257D843A25744
:1028C000A1076317F700A257DC43D843A257D8C328
:1028D000A257DC43DC473ED2A2473ED08257DC43BE
:1028E000D8438257D8C38257D8438257A10763176A
:1028F000F7008257DC43D8438257D8C38257DC4362
:10290000DC473ECEB25796073247BA97724798C314
:10291000B25796073247BA97724713074703D8C38F
:10292000B25796073247BA977247384798C7B25797
:1029300096073247BA971247D8C7B2579607324719
:10294000BA977247585798CB12478D47631BF700C9
:10295000F2479C5799C7B25796073247BA9709472B
:10296000D8C7B25796073247BA977247384BD8CB79
:10297000B25796073247BA9723AC0700F247945BE9
:10298000B257960732473304F70036850D20AA87E1
:10299000231EF400B25785073ED672479257E31DB7
:1029A000F7F2B2573E85F2506254216182800111E4
:1029B0002AC602CE39A0B24785073EC6F247850730
:1029C0003ECEB24703C707009307500AE305F7FE60
:1029D000F24789833ECEF247C207C1833E85056137
:1029E0008280011106CE2AC6B2479C5B3E85EF105D
:1029F00080493245EF1020490100F2400561828094
:102A0000411197E70100938767C09C439C4399E37A
:102A1000854711A0814781CB97E70100938787C540
:102A20007D5798C305A097E70100938727BE9C4375
:102A3000DC47DC473EC6B247D84397E7010093879F
:102A400067C398C3010041018280411197E70100EB
:102A5000938747A69C433EC6B2473E85410182808C
:102A6000411197E701009387A7BF9C4381E7854702
:102A70003EC619A897E70100938707C09C4381E7EA
:102A800089473EC611A002C6B2473E8541018280F9
:102A9000797106D62AC6B2473ECEB247F9C3F2478D
:102AA000D85797E701009387E7A09C43DC57637AE8
:102AB000F70AF2479C4F63CC070097E70100938722
:102AC000679F9C43DC5715471D8FF24798CFF2470D
:102AD000D44BF247D857BA878A07BA978A0717E7BD
:102AE00001001307E7A9BA976394F600854711A080
:102AF0008147A5C3F24791073E85EFD09FB597E781
:102B000001009387279B9C43D857F247D8D7F247B9
:102B1000D85797E70100938767B49C4363F9E700B0
:102B2000F247D85797E70100938747B398C3F24716
:102B3000D857BA878A07BA978A0717E70100130799
:102B400027A43E97F2479107BE853A85EFD0DFA5CF
:102B500009A897E701009387E7959C43D857F24768
:102B6000D8D70100B25045618280797106D62AC655
:102B7000B2473ECC02CEB247DDC397E70100938750
:102B800067939C4362476305F7007370043001A0AC
:102B9000E247FC4B81E77370043001A0E247FC4B35
:102BA0001387F7FFE247F8CBE247D857E247BC4B21
:102BB0006307F706E247FC4BBDE3E24791073E851A
:102BC000EFD03FA9E247B84BE247D8D7E247DC57FE
:102BD00015471D8FE24798CFE247D85797E7010086
:102BE0009387C7A79C4363F9E700E247D85797E765
:102BF00001009387A7A698C3E247D857BA878A07E8
:102C0000BA978A0717E70100130787973E97E247AD
:102C10009107BE853A85EFD03F9985473ECEF24772
:102C20003E85B250456182807370043097E70100A1
:102C3000938707A39C4391CF97E7010093878787EA
:102C40009C43F8430507F8C397E7010093878786FD
:102C50009C430100828097E70100938767A09C4313
:102C60008DCB97E701009387E7849C43FC4395C392
:102C700097E70100938707849C43F8437D17F8C3C7
:102C800097E70100938707839C43FC4399E37360B4
:102C9000043001008280411197E70100938787810A
:102CA0009C439C4F3EC697E701009387A7809C43B7
:102CB000D85797D701009387E77F9C439546338782
:102CC000E64098CFB2473E854101828097D7010008
:102CD0009387477E9C4389CB97D701009387877D55
:102CE0009C43F84B0507F8CB97D701009387877C67
:102CF0009C433E858280797106D62AC62EC42D3724
:102D000097D701009387077B9C43BC4FADE397D7D0
:102D100001009387277A9C430547F8CFA247A1CBB0
:102D200097D70100938707799C4391073E85EFD0A1
:102D30005F922247FD576310F70297D701009387F0
:102D400067779C439107BE8517E501001305458F02
:102D5000EFD09F8519A897E701009387E78F9C43E1
:102D60002247BA973ECE7245353CEFD02FEAE53583
:102D7000653D97D701009387E7739C43BC4F3ECCDA
:102D8000E2479DC3B24789CB97D7010093878772EB
:102D90009C4323AC070409A897D701009387877148
:102DA0009C43B84F7D17B8CF97D7010093878770A2
:102DB0009C4323AE07044535E2473E85B25045614A
:102DC0008280797106D62AC62EC432C236C0A93D89
:102DD00097D701009387076E9C43F84F8947630D8F
:102DE000F70697D701009387E76C9C43B44F3247AF
:102DF0001347F7FF758FB8CF97D701009387876B7D
:102E00009C430547F8CF8247A1CB97D70100938712
:102E1000676A9C4391073E85EFD0BF830247FD5709
:102E20006310F70297D701009387C7689C43910707
:102E3000BE8517E501001305A580EFD0EFF619A8B0
:102E400097E70100938747819C430247BA973ECC9E
:102E50006245893AEFD08FDBFD3BF933924789CB4E
:102E600097D70100938707659C43B84F924798C353
:102E700097D70100938707649C43F84F85476314F5
:102E8000F70002CE31A897D701009387A7629C4331
:102E9000B44F22471347F7FF758FB8CF85473ECE13
:102EA00097D70100938707619C4323AE07046533DE
:102EB000F2473E85B25045618280797106D62AC6B6
:102EC0002EC432C236C085473ECEB24781E773700A
:102ED000043001A0B2473ECC813B824789C7E2471C
:102EE000B84F824798C3E247FC4F3ECAE2470947C2
:102EF000F8CF1247914763EEE704924713972700F4
:102F000097D7010093878710BA97984397D7010006
:102F10009387C70FBA978287E247B84FA2475D8F62
:102F2000E247B8CF3DA0E247BC4F13871700E24706
:102F3000B8CF05A0E2472247B8CF21A8524789471A
:102F40006306F700E2472247B8CF21A002CE11A0C6
:102F5000010052478547631AF706E24791073E850D
:102F6000EFD02FEFE247D85797D701009387076F2D
:102F70009C4363F9E700E247D85797D7010093874E
:102F8000E76D98C3E247D857BA878A07BA978A0786
:102F900017D701001307C75E3E97E2479107BE852A
:102FA0003A85EFD06FE0E2479C5781C773700430D9
:102FB00001A0E247D85797D701009387A74F9C43BA
:102FC000DC5763F4E700EFD06FC47131F2473E8500
:102FD000B25045618280397106DE2ACE2ECC32CACB
:102FE00036C83AC685473ED6F24781E7737004304B
:102FF00001A0F2473ED4EFD04FCFAA873ED2C247BE
:1030000089C7A257B84FC24798C3A257FC4F3ED0BA
:10301000A2570947F8CF5247914763EEE704D247DA
:103020001397270097D70100938787FFBA97984394
:1030300097D701009387C7FEBA978287A257B84FE8
:10304000E2475D8FA257B8CF3DA0A257BC4F138770
:103050001700A257B8CF05A0A2576247B8CF21A842
:10306000025789476306F700A2576247B8CF21A0ED
:1030700002D611A0010002578547631DF708A25729
:103080009C5781C77370043001A097D701009387C4
:10309000A75E9C43A1EBA25791073E85EFD06FDB63
:1030A000A257D85797D701009387475B9C4363F992
:1030B000E700A257D85797D701009387275A98C39C
:1030C000A257D857BA878A07BA978A0717D7010035
:1030D0001307074B3E97A2579107BE853A85EFD05D
:1030E000AFCC11A8A257E107BE8517D50100130583
:1030F0006552EFD06FCBA257D85797D7010093876F
:10310000673B9C43DC5763F7E700B24781C7B24790
:10311000054798C392573E85EFD02FBCB2573E85E6
:10312000F25021618280797106D62AC62EC4B24738
:1031300081E77370043001A0B2473ECEEFD0EFBA02
:10314000AA873ECCF247FC4F3ECAF2470947F8CF68
:10315000F247BC4F13871700F247B8CF5247854755
:10316000631DF708F2479C5781C77370043001A0B4
:1031700097D70100938747509C43A1EBF2479107F3
:103180003E85EFD00FCDF247D85797D701009387F0
:10319000E74C9C4363F9E700F247D85797D7010003
:1031A0009387C74B98C3F247D857BA878A07BA970D
:1031B0008A0717D701001307A73C3E97F2479107EC
:1031C000BE853A85EFD04FBE11A8F247E107BE8514
:1031D00017D5010013050544EFD00FBDF247D857AE
:1031E00097D701009387072D9C43DC5763F7E700CF
:1031F000A24781C7A247054798C3E2473E85EFD063
:10320000CFAD0100B25045618280797106D62AC6E1
:10321000B2473ECCE24799E797D7010093878729C9
:103220009C4311A0E2473ECC0134E247F84F894766
:103230006318F700E24723AE070485473ECE11A08E
:1032400002CE113CF2473E85B250456182800111A9
:1032500006CE02C61D2B97D70100938727459C43B6
:103260009DC38148014881470947814613060040B4
:1032700097D50100938505DC170500001305051B94
:10328000EFE0AF852AC6B24781E77370043001A032
:10329000B2473E85F24005618280397106DE2ACE52
:1032A0002ECC32CA36C83AC6E24799E302D62DA8D8
:1032B0001305C002EF00302A2AD6B25795C7F12174
:1032C000B257724798C3B257624798CFB257524726
:1032D000D8CFB257424798D3B2573247D8D3B25714
:1032E00091073E85EFD04FABE24781E77370043022
:1032F00001A0B2573E85F25021618280397106DE0D
:103300002ACE2ECC32CA36C83AC602D6F24781E758
:103310007370043001A097D70100938727399C432D
:10332000B5CBE2473ED0D2473ED2F2473ED46247C9
:10333000954763C4E704EFF0AFF22A87894763102B
:10334000F70297D70100938767369C431810814690
:103350003246BA853E85EFD0AFE02AD625A897D76A
:1033600001009387A7349C43181081460146BA8513
:103370003E85EFD0EFDE2AD631A897D7010093879C
:10338000E7329C43181081464246BA853E85EFD00D
:103390000FF32AD6B2573E85F25021618280011187
:1033A0002AC6B2473ECEB24781E77370043001A00F
:1033B000F2479C433E8505618280797106D62AC614
:1033C0002EC497D701009387E72D9C43DC47DC4749
:1033D0003ECEF24791073E85EFD0AFA7F247D84FD8
:1033E0008547631BF702F247984FB247BA97B24638
:1033F0002246BE857245B9222A878547631EF7009B
:1034000001478146324681457245CD3D2ACCE2478F
:1034100081E77370043001A0F247DC537245829754
:103420000100B25045618280797106D62AC63C08F7
:103430003E8541282ACEE247BE8572451920692281
:10344000FDB7797106D62AC62EC4EFE06FF93C08A5
:103450003E8545282ACEE247B9EFA24799EB32478D
:10346000F24763E8E700EFE06FF9F2453245B13724
:10347000A9A0A24781CF97D701009387E7229C4359
:103480009C4393B7170093F7F70F3EC497D70100FB
:103490009387C72194433247F247B307F740224648
:1034A000BE853685EFD0FFDDEFE04FF5AA8791E7C7
:1034B000EFC0DFF519A0EFE06FF40100B2504561F5
:1034C000828001112AC697D701009387A71D9C43CC
:1034D0009C4393B7170093F7F70F3E87B24798C303
:1034E000B2479C4391EB97D701009387A71B9C435E
:1034F000DC479C433ECE11A002CEF2473E850561DB
:103500008280797106D62AC6EFE01F842ACE97D72B
:1035100001009387E7199C4372476377F700692A94
:10352000B247054798C321A0B24723A0070097D709
:1035300001009387E717724798C3F2473E85B25060
:1035400045618280797106D62AC62EC432C236C041
:1035500002CEB2472247D8C3B247324798CB224760
:10356000924763E8E702124782471D8FB2479C4F9C
:103570006365F70085473ECE99A097D701009387F2
:10358000A7129843B2479107BE853A85EFD0CF8501
:103590003DA0124782476379F7002247824763655F
:1035A000F70085473ECE21A897D701009387870F64
:1035B0009843B2479107BE853A85EFD0EF82F24734
:1035C0003E85B25045618280797106D6D9A0A24766
:1035D00063C0070CC2473ECEF247DC4B91C7F247AF
:1035E00091073E85EFD0EF865C003E85193F2ACCDF
:1035F000A2472547636FF7081397270097D7010065
:103600009387C7A3BA97984397D70100938707A3D7
:10361000BA9782873247F2479C4FBA973247BA86A9
:103620006246BE857245393F2A8785476313F70690
:10363000F247DC5372458297F247D84F8547631AA9
:10364000F7043247F2479C4FBA97014781463E86BE
:103650008145724565312ACAD24785EF73700430BF
:1036600001A03247F24798CFF2479C4F81E7737031
:10367000043001A0F247984FE247BA97E24662460B
:10368000BE857245C13531A07245EF00C07F11A0E3
:10369000010097D70100938767019C43380081465A
:1036A0000146BA853E85EFD06FD8AA87E39107F22D
:1036B0000100B25045618280797106D671A097D71A
:1036C0000100938727FE9C43DC479C433ECC97D761
:1036D0000100938727FD9C43DC47DC473ECAD24765
:1036E00091073E85EFC0FFF6D247DC5352458297E3
:1036F000D247D84F85476319F704D2479C4F62479A
:10370000BA973EC84247E24763F4E702D2474247CE
:10371000D8C3D247524798CB97D70100938787F8F1
:103720009843D2479107BE853A85EFC0FFEB29A8A1
:1037300001478146624681455245C9362AC6B2478D
:1037400081E77370043001A097D70100938787F554
:103750009C439C43ADF797D701009387A7F49C4304
:103760003ECE97D70100938727F4984397D701005F
:10377000938747F398C397D701009387E7F272477F
:1037800098C30100B25045618280411106C6EFF036
:10379000AFC997D70100938767F19C43C9E717D555
:1037A00001001305A5EDEFC0FFDB17D501001305E0
:1037B00025EEEFC03FDB97D701009387A7EE17D721
:1037C00001001307A7EB98C397D701009387C7EDB4
:1037D00017D701001307C7EB98C30146B145114540
:1037E000EFC07FF72A8797D70100938727EC98C30C
:1037F00097D70100938787EB9C4381E77370043070
:1038000001A097D70100938767EA9C4389CF97D798
:1038100001009387A7E99C4397D501009385858490
:103820003E85EFD05F9CEFF00FC30100B240410135
:103830008280797106D62AC6B2473ECEB24781E76A
:103840007370043001A0EFF02FBEF247DC4BB337AA
:10385000F00093F7F70F3ECCEFF0EFBFE2473E8565
:10386000B25045618280797106D62AC6B2473ECEF3
:10387000B24781E77370043001A0EFF0EFBAF2476E
:103880009C533ECCEFF02FBDE2473E85B2504561E0
:103890008280797106D62AC62EC4B2473ECEB24780
:1038A00081E77370043001A0EFF00FB8F2472247B0
:1038B00098D3EFF04FBA0100B250456182800111F8
:1038C00006CE714549292AC6B24789CBB24723A003
:1038D0000700B24791073E85EFC0DFC8B2473E857B
:1038E000F24005618280397106DE2AC62EC432C2DA
:1038F00036C0B2473ED402D21247B70700FFF98F55
:1039000081C77370043001A0924781E7737004305F
:1039100001A0EFF0EF94AA8799E3824799E38547E6
:1039200011A0814781E77370043001A0EFE04FAB35
:10393000A2579C433ED0A245324585240257A24758
:103940005D8F9247F98F12476310F7020257A24723
:10395000D98F3ED6A2579843924793C7F7FF7D8FE2
:10396000A25798C302C025A0824799CFA257938639
:1039700047001247B7070005D98F0246BE85368536
:10398000EFE03F8902D621A0A2579C433ED6EFE04C
:10399000EFA62ACE8247B1CBF24799E3EFC01FA72B
:1039A000EFF06FAF2AD63257B7070002F98F85EBD9
:1039B000EFF08FA7A2579C433ED632579247F98F1C
:1039C0001247631AF700A2579843924793C7F7FF2D
:1039D0007D8FA25798C3EFF00FA885473ED232578C
:1039E000B7070001FD17F98F3ED6B2573E85F2505A
:1039F000216182805D7186C62ACE2ECC32CA36C83D
:103A00003AC6F2473EDA02DC02D8F24781E7737029
:103A1000043001A06247B70700FFF98F81C77370B8
:103A2000043001A0E24781E77370043001A0EFF099
:103A30002F83AA8799E3B24799E3854711A081476D
:103A400081E77370043001A0EFE08F99D2579C4357
:103A50003ED64246E245325575242AD4A25799CF24
:103A6000B2573EDE02C6D247A9CBD2579843E247AF
:103A700093C7F7FF7D8FD25798C381A0B24781E7E4
:103A8000B2573EDE1DA8D24791C76257B707000163
:103A9000D98F3EDCC24791C76257B7070004D98F60
:103AA0003EDCD257938647006247E257D98F3246B1
:103AB000BE853685EFE0EFF502DEEFE02F942AD2E7
:103AC000B247B9CB925799E3EFC05F94EFF0AF9C48
:103AD0002ADE7257B7070002F98F8DEBEFF0CF9413
:103AE000D2579C433EDE4246E2457255212CAA87BE
:103AF00099CBD24789CBD2579843E24793C7F7FF78
:103B00007D8FD25798C3EFF00F9502D87257B70741
:103B10000001FD17F98F3EDEF2573E85B640616128
:103B20008280797106D62AC62EC4B2473ECEB247ED
:103B300081E77370043001A02247B70700FFF98FB7
:103B400081C77370043001A0EFF00F8EF2479C43E1
:103B50003ECCF2479843A24793C7F7FF7D8FF247C9
:103B600098C3EFF04F8FE2473E85B25045618280A7
:103B7000797106D62AC6B2473ECEEFC01F97AA87F4
:103B80003ECCF2479C433ECAE2473E85EFC0FF94DD
:103B9000D2473E85B250456182805D7186C62AC695
:103BA0002EC402DCB2473ED802DAB24781E7737016
:103BB000043001A02247B70700FFF98F81C7737057
:103BC000043001A0C25791073ED6B257A1073ED498
:103BD000EFE00F81B257DC473EDEC2579843A24761
:103BE0005D8FC25798C3BDA8F257DC433ED2F2574F
:103BF0009C433ED002DA0257B70700FFF98F3ECE52
:103C00000257B7070001FD17F98F3ED07247B7077B
:103C10000004F98F89EBC25798438257F98F89CFF7
:103C200085473EDA11A8C25798438257F98F025749
:103C30006314F70085473EDAD2579DC37247B70732
:103C40000001F98F89C762578257D98F3EDCC2576E
:103C50009843B7070002D98FBE857255EFE00FF980
:103C600092573EDE7257A257E310F7F8C2579843B7
:103C7000E25793C7F7FF7D8FC25798C3EFD01FF865
:103C8000C2579C433E85B64061618280797106D6F9
:103C90002AC6B2473ECEF24791073ECCEFD05FF442
:103CA0000DA0E247D847E247A1076315F7007370FC
:103CB000043001A0E247DC47B70500023E85EFE093
:103CC000EFF2E2479C43F1FF7245752AEFD01FF3F4
:103CD0000100B25045618280011106CE2AC62EC471
:103CE000A24532455D3D0100F2400561828001112F
:103CF00006CE2AC62EC4A245324525350100F24023
:103D00000561828001112AC62EC432C202CE9247BA
:103D100081EB3247A247F98F81CF85473ECE09A874
:103D20003247A247F98F22476314F70085473ECEFA
:103D3000F2473E850561828001112AC6B2473ECC1A
:103D4000B24799E302CE21A0E2479C4F3ECEF24714
:103D50003E8505618280397106DE2AC602D2EFD027
:103D60003FE8976703009387E7959C4381EB5522D3
:103D70009767030093870795054798C3B24789CF94
:103D8000A1473E87B247BA973EC6B2478D8B89C7D7
:103D9000B247F19B91073EC6B247F9CB3247E56780
:103DA000ED1763E7E70C976703009387A7903ED46E
:103DB00097670300938707909C433ED631A0B25784
:103DC0003ED4B2579C433ED6B257DC43324763F5EC
:103DD000E700B2579C43E5F7325797670300938794
:103DE000E78D6307F708A2579C432147BA973ED255
:103DF000B2579843A25798C3B257D843B247B307B4
:103E0000F740214706076378F7043257B247BA975D
:103E10003ECEB257D843B2471D8FF247D8C3B257F0
:103E20003247D8C3F247DC433ECC97670300938701
:103E300067883ED021A082579C433ED082579C4346
:103E4000DC436247E3E9E7FE82579843F24798C3B1
:103E50008257724798C397C701009387E7669843D4
:103E6000B257DC431D8F97C701009387E76598C35E
:103E7000EFD0DFD8925799E3EF00103292573E858A
:103E8000F25021618280797106D62AC6B2473ECCB3
:103E9000B247BDC3A147B307F0406247BA973ECCD3
:103EA000E2473ECAEFD0DFD3D247DC433EC8976734
:103EB0000300938727803ECE21A0F2479C433ECE4D
:103EC000F2479C43DC434247E3E9E7FEF24798436D
:103ED000D24798C3F247524798C3D247D84397C7AF
:103EE00001009387675E9C433E9797C701009387C5
:103EF000A75D98C3EFD09FD00100B250456182808A
:103F000097C701009387475C9C433E8582800100F0
:103F10008280411197C701009387077AF19B3EC6C3
:103F20009757030093870779324798C39757030041
:103F30009387477823A20700975703009387077852
:103F400065677117D8C3975703009387277723A016
:103F50000700B2473EC4A24765677117D8C3A2479E
:103F6000175703001307877598C30100410182802A
:103F700001112AC62EC432C2A2473ECEB2473ECC61
:103F80003247A247D98F8D8BA1E319A8F2479843F6
:103F9000E24798C3E24791073ECCF24791073ECEF5
:103FA0009247F5173247BA976247E361F7FE29A8AF
:103FB0007247930717003ECEE2479386170036CC30
:103FC000034707002380E70032479247BA976247CA
:103FD000E360F7FEB2473E850561828001112AC683
:103FE0002EC432C232479247D98F8D8B9DEFA247A4
:103FF00093F7F70F3ECAD247A2075247D98F3ECA5E
:10400000D247C2075247D98F3ECAB2473ECE39A0E7
:10401000F247138747003ACE524798C33247924738
:10402000BA977247E366F7FE1DA0B2473ECC11A8CF
:10403000E247138717003ACC22471377F70F238004
:10404000E70032479247BA976247E363F7FEB24709
:104050003E850561828001112AC6B2473ECE21A06D
:10406000F24785073ECEF24783C70700F5FB72474C
:10407000B247B307F7403E850561828001112AC629
:104080002EC4B247138717003AC683C70700A30F91
:10409000F100A247138717003AC483C70700230F14
:1040A000F1008347F10199C70347F1018347E1011B
:1040B000E309F7FC0347F1018347E101B307F74048
:1040C0003E850561828001112AC62EC4B2473ECECC
:1040D00001002247930717003EC4F247938617005A
:1040E00036CE034707002380E70083C70700F5F3B8
:1040F000B2473E850561828001112AC602CE02CCFC
:1041000021A0B24785073EC6B24703C70700930701
:104110000002E308F7FEB24703C707009307D00287
:104120006309F700B24703C707009307B0026311A2
:10413000F704B24783C70700938737FD93B717008B
:1041400093F7F70F3ECCB24785073EC615A07247DE
:10415000BA878A07BA9786073ECEB24713871700F9
:104160003AC683C70700938707FD7247BA973ECECA
:10417000B24783C70700E1FFE24789C7F247B307A9
:10418000F04011A0F2473E850561828001112AC6E8
:1041900097570300938707579C4393861700175739
:1041A00003001307275614C332471377F70F9756A8
:1041B000030093862659B6972380E7003247A94724
:1041C000630BF700975703009387C75398439307F0
:1041D00000046315F704975703009387A7563ECE54
:1041E00005A8F247138717003ACE03C70700B707A1
:1041F00010F0938707F098C3975703009387875071
:104200009C431387F7FF975703009387A74F98C3E3
:10421000975703009387074F9C43E1F781473E85FB
:10422000056182804D7123261114232481142322D9
:10423000911423202115232E3113232C4113232ADB
:1042400051132ACE2ECC32C836CA3AC63EC442C218
:1042500023260112B2473E8A814AC24752485286FB
:10426000D6863E85C285EF10E040AA872E883E861E
:10427000C2868327C112138717002326E1123287D3
:104280008A07141AB69723AEE7EEB2473E848144FC
:10429000D247268763E8E702D24726876396E7007E
:1042A000C247228763E0E702B2473E8981494A86D6
:1042B000CE864245D245EF00305EAA872E883EC8A2
:1042C00042CA49BF010029A0F247E2451245829740
:1042D000A2471387F7FF3AC40327C112E346F7FE4C
:1042E00025A88327C1128A07181ABA9703A7C7EF10
:1042F0008327C1128A07141AB69783A6C7EFA5476A
:1043000063F5D7009307700519A093070003BA97C8
:104310007247E2453E8502978327C1121387F7FF54
:104320002326E112E34FF0FA01008320C114032495
:10433000811483244114032901148329C113032AFE
:104340008113832A41137161828041112AC62EC4D0
:10435000A2460547635ED700B2479C439D07E19B99
:1043600093868700324714C303A847009C4335A0B7
:10437000224719CB3247184313064700B24690C272
:104380001843BA87014811A832471843130647005B
:10439000B24690C21843BA8701483E85C2854101A2
:1043A000828041112AC62EC4A2460547635ED7000B
:1043B000B2479C439D07E19B93868700324714C315
:1043C00003A847009C4305A8224701CF3247184362
:1043D00013064700B24690C21843BA877D873A88D1
:1043E00019A83247184313064700B24690C2184333
:1043F000BA877D873A883E85C285410182803971BE
:1044000006DE22DC26DA2AC62EC432C236C011A845
:1044100063070424924785073EC2B247A24522851E
:104420008297924783C707003E8493075002E311A7
:10443000F4FE924785073EC292473EC893070002AA
:10444000A30BF100FD573ECEFD573ECC02D0924764
:10445000138717003AC283C707003E849307D4FD31
:10446000130750056364F71E1397270097C70100D1
:10447000938747C0BA97984397C70100938787BF30
:10448000BA9782879307D002A30BF100C9B79307AD
:104490000003A30BF10065BF02CC6247BA878A070D
:1044A000BA978607A297938707FD3ECC924783C7AA
:1044B00007003E849307F00263D6870293079003B8
:1044C00063C28702924785073EC2C1BF82471387F6
:1044D00047003AC09C433ECC39A0F247E3D907F6E7
:1044E00002CEB5B70100F247E3D307F6E2473ECE6E
:1044F000FD573ECCA9BF825785073ED089BF824772
:10450000138747003AC09C433247A2453E85029735
:10451000B1A28247138747003AC0844389E497C415
:1045200001009384A4B4F2476357F0040347710178
:104530009307D0026301F704E247BE852685EF00AA
:1045400070332A87F247998F3ECE11A883477101B5
:104550003247A2453E850297F247FD173ECEF2470D
:10456000E346F0FE09A8B247A2452285829785045A
:10457000F247FD173ECE83C704003E841DC0E247CC
:10458000E3C307FEE247FD173ECCE247E3DD07FC4D
:1045900009A8B247A245130500028297F247FD170A
:1045A0003ECEF247E347F0FE55A88A8782553E8506
:1045B000CD3BAA872E883ED442D6A2573258C28716
:1045C00063D90702B247A2451305D0028297A255CC
:1045D000325681470148B386B740368533B5A700C8
:1045E0003307C840B307A7403E87B6873A883ED412
:1045F00042D6A9473ED21DA8A9473ED215A0A14741
:104600003ED239A885473ED0B247A24513050003E4
:104610008297B247A245130580078297C1473ED2D1
:104620008A8782553E8515332AD42ED61257834762
:1046300071013E88F2472256B256A2453245DD3618
:1046400031A8B247A2452285829709A8B247A24560
:10465000130550028297C2473EC20100D9B3010040
:10466000F2506254D2542161828041112AC6B707A8
:1046700010F0938707F2324798C301A05D7106D608
:104680002AC62EDA32DC36DEBAC0BEC2C2C4C6C604
:104690009C0891173ECEF247BE86324681451705EB
:1046A00000001305E5AEA13B81473E85B250616134
:1046B000828001112AC62EC41EC2A2473ECEF247F6
:1046C0009C4332471377F70F2380E700F2479C4360
:1046D00013871700F24798C30100056182801D719E
:1046E00006DE2AC62EC4B2C4B6C6BAC8BECAC2CC7A
:1046F000C6CE9C103ED25C084C081706000013067C
:1047000086FB7D779346F7FF0565130505803388A3
:10471000A5003378E8001368783B23A007013295A1
:10472000698F13677733D8C333F7D50093154701E3
:1047300037870300130737394D8F98C73377D60073
:10474000931647013707030013077706558FD8C71D
:104750000F100000B2473ED69C10A1173ED422573E
:104760005C083E857C00BA862246BE854939B24740
:1047700023800700B2473E87B257B307F7403E8514
:10478000F250256182804111370510F0130545F480
:1047900008412AC6370510F0130505F408412AC45C
:1047A000370510F0130545F40841B248E39EA8FC14
:1047B00032452A8381431317030081462245AA8587
:1047C0000146B3E7B6003368C700370710F013059A
:1047D00087F48565938505FA0146B386B700B688E8
:1047E000B3B8F8003307C800B387E8003E87B68740
:1047F0003A881CC123220501010041018280411138
:1048000006C651379307000873A047300100B24035
:1048100041018280011106CE2AC617C50100130589
:10482000E59AEFF0BFE50100F240056182800111D9
:1048300006CE2AC617C501001305C599EFF01FE47F
:104840000100F24005618280797106D62AC602CE47
:1048500029A00100F24785073ECE724785679387FE
:104860007738E3D8E7FE17C5010013052597EFF069
:10487000FFE0F1BF411106C60145152A0100B24013
:1048800041018280011106CE02C6EF0060792A87BD
:104890008547630CF70017C501001305A594EFF0D9
:1048A000FFDDB24793E727003EC6B2473E85F240A0
:1048B00005618280011106CE02C66D3F1707000018
:1048C00013076704814605469305200317C50100B9
:1048D0001305C592EFE07F9C2AC6B24799CBEFD073
:1048E000AFC6AA87014781463E8685453245EFE03F
:1048F000FFA002C4EFD0EFA481473E85F2400561DE
:104900008280797106D62AC697C701009387C7BAF5
:104910009C431387470697C701009387E7B998C35D
:1049200097C70100938787B99C431387470697C7AA
:1049300001009387A7B898C397C701009387C7B7AB
:1049400098439307F07C63D3E70497C701009387EC
:10495000A7B69C431387078397C701009387C7B502
:1049600098C30D372ACEF24799EB97C7010093877A
:10497000E7B4984385679387F77663DBE700F247F0
:104980003E85EFF09FCEEFD0AFA321A0010011A094
:104990000100B250456182807370043001A00100B3
:1049A000828041112AC62EC47370043001A0011107
:1049B00006CE2AC6814801488147324797560300F0
:1049C000938646DC1306004097C501009385058455
:1049D000170500001305C508EFC03F908148014846
:1049E00081473247975603009386E6D91306004065
:1049F00097C5010093850582170500001305451B27
:104A0000EFC0BF8D81480148814732479756030068
:104A1000938686D71306004097C5010093850580CD
:104A20001705000013050533EFC03F8B814801488F
:104A30008147324797560300938626D513060040D8
:104A400097B501009385057E1705000013050547FE
:104A5000EFC0BF880100F240056182805D7186C6AB
:104A6000A2C4A6C2CAC02AC6231F010297B701006A
:104A70009387C77B03A847009C433EC842CAB247FE
:104A80003EDC97B701009387E77A03A847009C4371
:104A90003ED842DA97B701009387477A03A84700C8
:104AA0009C433ED442D697B701009387A77903A8C9
:104AB00047009C433ED042D2C2575258A25632576A
:104AC0003686BA863E85C285EF10C00AAA872E8830
:104AD0003E85C285825712583E86C286EF20802AC4
:104AE000AA872E883ECC42CEE2477248C246524741
:104AF0003686BA863E85C285EF20D017AA872E88D3
:104B0000014681463E85C285EF200018AA8763D5FD
:104B10000704E24772483E8437070080B344E80048
:104B2000C24752483E86C2862285A685EF20901451
:104B3000AA872E883E85C285054997B701009387CD
:104B4000E7709043D443EF206004AA876343F000EA
:104B500001499377F90F35A8E2477248C246524798
:104B60003686BA863E85C285EF20D010AA872E8869
:104B70003E85C285054997B701009387276D90430D
:104B8000D443EF20A000AA876343F0000149937744
:104B9000F90F81C78547231FF1028317E103E392D1
:104BA00007EEE25705472390E700E1BD5D7186C639
:104BB000A2C4A6C2CAC02AC6231F010297B7010019
:104BC0009387476903A847009C433ED842DA97B7CA
:104BD00001009387A76803A847009C433ED442D6B0
:104BE00097B701009387076803A847009C433ED00E
:104BF00042D2C2575258A25632573686BA863E859E
:104C0000C285EF10A077AA872E883E85C28582577D
:104C100012583E86C286EF20E016AA872E883EC82C
:104C200042CAB2473EDC97B701009387A76203A848
:104C300047009C433ED842DA97B70100938707624A
:104C400003A847009C433ED442D697B70100938700
:104C5000676103A847009C433ED042D2C2575258D6
:104C6000A25632573686BA863E85C285EF1000714D
:104C7000AA872E883E85C285825712583E86C286F4
:104C8000EF204010AA872E883ECC42CEE2477248E1
:104C9000C24652473686BA863E85C285EF20807D61
:104CA000AA872E88014681463E85C285EF10D07DB9
:104CB000AA8763D50704E24772483E84370700801D
:104CC000B344E800C24752483E86C2862285A68584
:104CD000EF20407AAA872E883E85C285054997B77E
:104CE00001009387A7569043D443EF10306AAA87F8
:104CF0006343F00001499377F90F35A8E247724802
:104D0000C24652473686BA863E85C285EF208076F7
:104D1000AA872E883E85C285054997B701009387EB
:104D2000E7529043D443EF107066AA876343F000C4
:104D300001499377F90F81C78547231FF102831734
:104D4000E103E39207EEE25705472390E700E1BD58
:104D50005D7186C6A2C42AC6A9473EDA231D010298
:104D6000B2473ED8D2578E073E85EFE0DFFE2AD607
:104D700002D002D202CC02CE02DE95A07255EF2004
:104D80003071F2578E0732573304F70097B701009E
:104D90009387C74D9043D443EF00D05DAA872E88F8
:104DA0001CC0232204017255EF20906E97B70100BA
:104DB0009387C74B9043D443EF00D05BAA872E88DC
:104DC0003E85C285825712583E86C286EF00905AB1
:104DD000AA872E883ED042D2F25785073EDE725710
:104DE000D257E36DF7F802DE3DA0F2578E07325737
:104DF000BA9703A847009C43E24672473686BA86B4
:104E00003E85C285EF001057AA872E883ECC42CE41
:104E1000F25785073EDE7257D257E368F7FC825798
:104E20001258E24672473686BA863E85C285EF2022
:104E30006064AA872E883EC842CAC24752480146CB
:104E400081463E85C285EF103064AA8763D607028B
:104E5000C2475248054417B701001307A741104342
:104E600054433E85C285EF103062AA8763C30700B2
:104E700001449377F40F25A0C2475248054417B761
:104E800001001307A73C104354433E85C285EF1031
:104E9000F04FAA876343F00001449377F40F81C772
:104EA0008547231DF1028317A103E39307ECC25743
:104EB00005472390E7006DBD5D7186C6A2C42AC672
:104EC000A9473EDA231D0102B2473ED8D2578E07CA
:104ED0003E85EFE05FE82AD602D002D202CC02CEB5
:104EE00002DE95A07255EF20B05AF2578E07325766
:104EF0003304F70097B70100938747389043D443B2
:104F0000EF105068AA872E881CC023220401725516
:104F1000EF20105897B70100938747369043D4434A
:104F2000EF105066AA872E883E85C2858257125898
:104F30003E86C286EF001044AA872E883ED042D219
:104F4000F25785073EDE7257D257E36DF7F802DE5F
:104F50003DA0F2578E073257BA9703A847009C43EB
:104F6000E24672473686BA863E85C285EF0090409B
:104F7000AA872E883ECC42CEF25785073EDE725776
:104F8000D257E368F7FC82571258E24672473686DA
:104F9000BA863E85C285EF20E04DAA872E883EC89E
:104FA00042CAC2475248014681463E85C285EF103B
:104FB000B04DAA8763D60702C2475248054417B7C7
:104FC00001001307272B104354433E85C285EF1081
:104FD000B04BAA8763C3070001449377F40F25A061
:104FE000C2475248054417B701001307272610434C
:104FF00054433E85C285EF107039AA876343F000A1
:1050000001449377F40F81C78547231DF10283176D
:10501000A103E39307ECC25705472390E7006DBD5A
:10502000411185473EC602C435A817470300130740
:105030006775A2478607BA9783D7070013970701BA
:10504000418385476304F70002C611A81747030090
:1050500013074773A2478607BA9723900700A24712
:1050600085073EC422478D47E3D1E7FCB2473E8522
:1050700041018280B305B500930705006386B70040
:1050800003C70700631607003385A7406780000049
:10509000938717006FF09FFE130101FD23229102F9
:1050A000232A5101232611022324810223202103D4
:1050B000232E3101232C4101232861012326710174
:1050C00023248101232291012320A101930A0500B9
:1050D00093840500639E06381304060093090500B7
:1050E00017B901001309892163F8C512B707010038
:1050F000138B05006378F6101307F00F3337C700E2
:1051000013173700B357E6003309F9008346090047
:105110003387E60093060002B386E640638C060000
:10512000B394D40033D7EA003314D600336B97001E
:10513000B399DA00935A040193850A0013050B0012
:10514000EF2090461309050093850A00931B040184
:1051500013050B00EF20D04093DB0B0193040500F7
:105160009305050013850B00EF20D03C13190901AE
:1051700093D70901B367F900138A040063FEA700FF
:10518000B3878700138AF4FF63E8870063F6A700FC
:10519000138AE4FFB3878700B384A74093850A008E
:1051A00013850400EF2050401309050093850A0081
:1051B00013850400EF20D03A939909019304050068
:1051C000930505001319090113850B0093D90901F3
:1051D000EF205036B36939011386040063FCA9003F
:1051E000B30934011386F4FF63E6890063F4A90070
:1051F0001386E4FF13140A013364C400130A000089
:105200006F000013B707000113070001E36CF6EE0F
:10521000130780016FF01FEF138A0600631A060060
:105220009305000013051000EF20903313040500D0
:10523000B7070100637EF4129307F00F63F4870051
:10524000130A8000B35744013309F90003470900EA
:105250009306000233074701B386E64063940612C3
:10526000B3848440130A1000135B040193050B0000
:1052700013850400EF2050331309050093050B003C
:1052800013850400931B0401EF20902D93DB0B0189
:10529000930405009305050013850B00EF2090296A
:1052A0001319090193D70901B367F900938A040020
:1052B00063FEA700B3878700938AF4FF63E8870043
:1052C00063F6A700938AE4FFB3878700B384A740FF
:1052D00093050B0013850400EF20102D1309050022
:1052E00093050B0013850400EF2090279399090183
:1052F00093040500930505001319090113850B009C
:1053000093D90901EF201023B369390113860400F2
:1053100063FCA900B30934011386F4FF63E6890036
:1053200063F4A9001386E4FF13940A013364C400F4
:105330001305040093050A008320C102032481029F
:1053400083244102032901028329C101032A810127
:10535000832A4101032B0101832BC100032C81000F
:10536000832C4100032D010013010103678000001D
:10537000B7070001130A0001E366F4EC130A800189
:105380006FF05FEC3314D40033DAE400B399DA0041
:1053900033D7EA00935A0401B394D40093850A00EA
:1053A00013050A00336B9700EF2010201309050046
:1053B00093850A0013050A00931B0401EF20501A7D
:1053C00093DB0B01930405009305050013850B0087
:1053D000EF2050161319090113570B013367E90029
:1053E000138A0400637EA70033078700138AF4FF43
:1053F000636887006376A700138AE4FF330787009A
:10540000B304A74093850A0013850400EF20D01948
:105410001309050093850A0013850400EF2050143A
:10542000930405009305050013850B00EF209010F1
:1054300013170B011357070113190901B367E9008B
:105440001387040063FEA700B38787001387F4FF68
:1054500063E8870063F6A7001387E4FFB38787003C
:10546000131A0A01B384A740336AEA006FF0DFDF42
:1054700063ECD51EB707010063F4F6041307F00FC1
:10548000B335D7009395350033D7B60097B70100F1
:105490009387C7E6B387E70003C70700130A000234
:1054A0003307B700330AEA4063160A0213041000F8
:1054B000E3E096E833B6CA00134416006FF05FE7E6
:1054C000B707000193050001E3E0F6FC93058001B6
:1054D0006FF09FFBB35CE600B3964601B3ECDC00D3
:1054E00033D4E40093DB0C01B397440133D7EA00D3
:1054F00093850B0013050400336BF700B3194601C5
:10550000EF20900A1309050093850B001305040092
:10551000139C0C01EF20D004135C0C0193040500D4
:105520009305050013050C00EF20D00013190901A5
:1055300013570B013367E90013840400637EA7004F
:10554000330797011384F4FF636897016376A7001C
:105550001384E4FF33079701B304A74093850B003E
:1055600013850400EF2050041309050093850B00F8
:1055700013850400EF20C07E930405009305050009
:1055800013050C00EF20007B93170B011319090181
:1055900093D70701B367F9001386040063FEA700E1
:1055A000B38797011386F4FF63E8970163F6A700BA
:1055B0001386E4FFB387970113140401B70B0100AE
:1055C0003364C4001389FBFF337D240133F92901BF
:1055D000B384A7409305090013050D00EF208075E3
:1055E000935C040193050900130B050013850C005F
:1055F000EF20407493D90901130C0500938509002D
:1056000013850C00EF200073130905009385090032
:1056100013050D00EF2000723305850193570B0130
:105620003385A70063748501330979019357050118
:10563000B387270163E6F402E392F4BCB7070100E5
:105640009387F7FF3375F50013150501337BFB00D6
:1056500033964A0133056501130A0000E37AA6CCAC
:105660001304F4FF6FF09FB9130A00001304000045
:105670006FF01FCC130101FB23248104232291042A
:10568000232E3103232291032326110423202105F5
:10569000232C4103232A510323286103232671036A
:1056A000232481032320A103232EB101930C0500A1
:1056B000938905001304050093840500639E062664
:1056C00013090600138A060097BA0100938A0AC3D9
:1056D00063F4C514B70701006376F6129307F00F61
:1056E00063F4C700130A8000B3574601B38AFA0077
:1056F00003C70A001305000233074701330AE540D8
:10570000630C0A00B395490133D7EC003319460105
:10571000B364B70033944C01935A090193850A008E
:1057200013850400EF2040689309050093850A0063
:10573000131B090113850400EF208062135B0B012A
:105740009305050013050B00EF20C05E9399090136
:1057500093570401B3E7F90063FAA700B387270161
:1057600063E6270163F4A700B3872701B384A7404A
:1057700093850A0013850400EF2000639309050058
:1057800093850A0013850400EF20805D1314040143
:10579000930505009399090113050B0013540401A7
:1057A000EF20405933E48900637AA40033042401D4
:1057B000636624016374A400330424013304A44009
:1057C00033554401930500008320C1040324810460
:1057D00083244104032901048329C103032A81038B
:1057E000832A4103032B0103832BC102032C810273
:1057F000832C4102032D0102832DC10113010105F8
:1058000067800000B7070001130A0001E36EF6ECA1
:10581000130A80016FF05FED631A06009305000024
:1058200013051000EF20C05313090500B70701004E
:10583000637AF90E9307F00F63F42701130A8000CF
:10584000B3574901B38AFA0003C70A0013050002DF
:10585000B384294133074701330AE540E30E0AEADE
:1058600033194901B3DAE900B395490133D7EC00A4
:1058700093540901336BB70013850A009385040024
:10588000EF2080529309050093850400931B0901C2
:1058900013850A00EF20C04C93DB0B019305050034
:1058A00013850B00EF2000499399090193570B01D1
:1058B000B3E7F90033944C0163FAA700B3872701DB
:1058C00063E6270163F4A700B3872701B38AA740E3
:1058D0009385040013850A00EF20004D930905000D
:1058E0009385040013850A00EF2080479305050087
:1058F00013850B00EF20004493150B0193990901C8
:1059000093D50501B3E5B90063FAA500B385250178
:1059100063E6250163F4A500B3852501B384A540A2
:105920006FF09FDFB7070001130A0001E36AF9F087
:10593000130A80016FF0DFF0E3E8D5E8B707010054
:1059400063FCF604930BF00F33B5DB001315350041
:1059500033D7A60097B701009387479AB387E7002C
:1059600083CB070093050002B38BAB00338B7541EB
:10597000631E0B0263E4360163EACC003384CC403F
:10598000B386D94033B58C00B384A6401305040018
:10599000938504006FF05FE3B70700011305000172
:1059A000E3E8F6FA130580016FF09FFAB3966601FB
:1059B000335D7601336DDD0033D47901B395690130
:1059C00033DC7C0193540D01336CBC0013050400DF
:1059D00093850400B31A6601EF20003D130A050009
:1059E000938504001305040033996C01931C0D0189
:1059F000EF20003793DC0C0113040500930505002C
:105A000013850C00EF200033131A0A0113570C0101
:105A10003367EA00130A0400637EA7003307A70177
:105A2000130AF4FF6368A7016376A700130AE4FF73
:105A30003307A701B309A740938504001385090024
:105A4000EF208036938504001304050013850900B8
:105A5000EF200031930505009304050013850C0029
:105A6000EF20402D93150C011314040193D505016B
:105A7000B365B4001387040063FEA500B385A501D8
:105A80001387F4FF63E8A50163F6A5001387E4FF1D
:105A9000B385A501131A0A01B70C0100336AEA00A5
:105AA0001384FCFFB3778A0033F48A00B384A540E3
:105AB00013850700930504002326F100135A0A01F9
:105AC000EF204027930905009305040013050A0001
:105AD000EF20402613DC0A01930D050093050C000E
:105AE00013050A00EF2000258327C100130A0500D3
:105AF00093050C0013850700EF20C0233305B50183
:105B000013D709013307A7006374B701330A9A0159
:105B1000B70701009387F7FF935507013377F70025
:105B200013170701B3F7F900B3854501B307F70071
:105B300063E6B400639EB400637CF900338657418A
:105B4000B3B7C700B385A541B385F54093070600F9
:105B5000B307F9403339F900B385B440B385254123
:105B600033947501B3D767013365F400B3D565018C
:105B70006FF09FC5370810001308F8FF130101FEEE
:105B8000B378B80013D745019357D50123282101D5
:105B90001379F77F139738003378D800B3E7E7001D
:105BA00013D7460113183800232A91001377F77F83
:105BB00093D8F601232E11009356D601232C810091
:105BC0002326310193D4F50133E306011315350083
:105BD000131636003308E9406394143B6354001FE6
:105BE000631207143367C3006314070C9306F07F36
:105BF00013070800631CD830B3E6A700639806308B
:105C000093070000130500009396870063DE0600EB
:105C1000130717009306F07F630CD774B70680FF55
:105C20009386F6FFB3F7D7009396D7011355350047
:105C300033E5A6009306F07F93D73700631ED700A5
:105C40003365F5009307000063080500B7070800F7
:105C50001305000093040000B70610009386F6FFBA
:105C6000B3F7D700B70610801377F77F9386F6FF58
:105C700013174701B3F7D700B3E7E70037070080F2
:105C80001347F7FF8320C101032481019395F40199
:105C9000B3F7E70033E7B70083244101032901018B
:105CA0008329C100930507001301010267800000EA
:105CB0009305F8FF639C05043306C5003335A60041
:105CC000B3876700B387A70013071000130506000A
:105CD0009396870063DC0622130717009306F07F74
:105CE000E300D7F2B70680FF9386F6FFB3F6D7003E
:105CF00093551500137515009397F60133E5A5002C
:105D000033E5A70093D716006F0040201307F07FFC
:105D10006314E80233E7A700630007621307F07F0C
:105D20006F00C01E1307F07FE306E9FE370780000F
:105D30003363E3009305080013078003634EB7063F
:105D40001307F0016342B704130700023307B7409B
:105D5000B356B6003318E3003316E6003368D800B4
:105D60003336C0003368C800B355B3003308A80009
:105D7000B385F500B337A800B387F5001305080015
:105D8000130709006FF0DFF4130700023358B30064
:105D9000930600006388E50093060004B385B640CF
:105DA000B316B30033E6C6003336C0003368C8000C
:105DB000930500006FF09FFB3368C3003338000188
:105DC0006FF01FFF630A080E631E0908B3E6A70001
:105DD000639206029307F07F6318F7003365C300F0
:105DE00093070000E30205E2930703001305060092
:105DF0006F00C0119306F0FF631CD8003305C50087
:105E0000B38767003336C500B387C7006FF05FEC18
:105E10009306F07F1348F8FFE302D7FC9306800354
:105E200063C606099306F00163CA060593050002DE
:105E3000B3850541B3580501B396B7003315B500D6
:105E4000B3E616013335A00033E5A60033D80701C9
:105E50003305C50033086800B337C500B307F80041
:105E60006FF01FE79306F07FE30AD7F6B7068000CE
:105E700033080041B3E7D7006FF05FFA93080002E0
:105E8000B3D60701930500006308180193050004C9
:105E900033880541B395070133E5A5003335A000EC
:105EA00033E5A600130800006FF09FFA33E5A70062
:105EB0003335A0006FF01FFF130719009375F77FAC
:105EC0009306100063C8B60833E7A70063140906F9
:105ED00063080744B366C300130700006388060223
:105EE0003306C5003335A600B3876700B387A70024
:105EF000939687001305060063DA0600370780FFD4
:105F00001307F7FFB3F7E700130710009376750048
:105F1000E38C06CE9376F50013064000E386C6CEEA
:105F20009306450033B5A600B387A7001385060086
:105F30006FF09FCD630C073E3368C300E30008DEBB
:105F4000B7074000130500001307F07F930400001B
:105F50006FF09FCB9306F07FE304D7CA3306C500EA
:105F600033886700B337A6003308F8001315F8012B
:105F7000135616003365C500935718006FF01FF9CC
:105F8000635E000F6312070A3367C300E30007C6AE
:105F90009306F8FF639E06023306C5403335C500FD
:105FA000B3876740B387A7401307100013050600A7
:105FB00093968700E3DC06F4370480001304F4FFB3
:105FC00033F4870093090500130907006F000027C9
:105FD0001307F07FE300E8D413078003634AD70870
:105FE0001307F001634ED704130700023307D740AD
:105FF000B355D6003318E3003316E6003368B80013
:106000003336C0003368C800B356D30033080541A7
:10601000B386D740B3370501B387F64013050800B0
:10602000130709006FF0DFF81307F07FE304E9CEF0
:10603000370780003363E300930608006FF0DFF951
:10604000130700023358D300130400006388E600EE
:1060500013040004B306D4403314D3003366C400E1
:106060003336C0003368C800930600006FF01FFA93
:106070003368C300333800016FF01FFF630A080E56
:10608000631E0908B3E6A700639006029307F07F3A
:106090006316F7003365C3006308052A93070300FE
:1060A000130506006F00C00F9306F0FF631ED800B3
:1060B0003305A640B307F3403336A600B387C74085
:1060C000938408006FF0DFEE9306F07F1348F8FF2B
:1060D000E302D7FC9306800363C606099306F0012A
:1060E00063CA060593050002B3850541335E0501C9
:1060F000B396B7003315B500B3E6C6013335A0003B
:1061000033E5A60033D807013305A6403308034121
:10611000B337A600B307F8406FF09FFA9306F07FFD
:10612000E30AD7F6B706800033080041B3E7D7008B
:106130006FF05FFA130E0002B3D60701930500005B
:106140006308C8019305000433880541B39507012E
:1061500033E5A5003335A00033E5A60013080000A1
:106160006FF09FFA33E5A7003335A0006FF01FFFF3
:10617000130719001377F77F9306100063CAE60828
:10618000B3E6A7003367C30063140906639E0600E5
:106190006302071C930703001305060013070000A2
:1061A000938408006FF09FD663000704B306C540D0
:1061B000B335D500338767403307B7409315870061
:1061C00063DC05003305A640B307F3403336A60071
:1061D000B387C7406FF09FFC33E5E600630A050C08
:1061E0009307070013850600130700006FF01FD206
:1061F000639C060063080716930703001305060057
:10620000938408006FF09FB1E30A07B06FF05FD38B
:10621000B309C54033846740333835013304044142
:106220001317840063520708B309A6403304F340F0
:10623000B33736013304F44093840800630E040638
:1062400013050400EF10903C130785FF9307F0013E
:1062500063CCE70693070002B387E7403314E400FA
:10626000B3D7F90033E487003395E9006340270B87
:1062700033072741930717009306F00163CEF60416
:10628000130700023307F7403356F500B316E40056
:106290003315E500B3E6C6003335A00033E5A600AC
:1062A000B357F4006FF05FF433E58900E31805F8A5
:1062B000930700006F00800A13850900EF10103566
:1062C000130505026FF05FF8130485FD3394890010
:1062D000130500006FF09FF9130717FE1306000265
:1062E0003357E400930600006388C7009306000458
:1062F000B386F640B316D4003365D5003335A0001D
:106300003365A700930700006FF01FEEB70780FF0B
:106310009387F7FF3307E940B377F4006FF01FBFAF
:1063200093070300130506006FF01FEC93070300AB
:10633000130506006FF09F9E9307000013050000F1
:106340001307F07F6FF05F8C9307000093840800C1
:106350006FF09F8B930700001305000013070000E8
:106360006FF0DFBE13050000B70740006FF0DFBD20
:1063700093070000130500006FF01F8B130101FB52
:1063800023248104232C41033704100013DA450130
:1063900023202105232E3103232A510323248103A3
:1063A0001304F4FF232611042322910423286103FC
:1063B00023267103232291032320A103232EB1015D
:1063C000137AFA7F13090500130C0600938A06005E
:1063D0003374B40093D9F50163060A0A9307F07F7A
:1063E0006304FA1013143400B70780003364F40018
:1063F000135BD501336B8B0093143500130A1AC05D
:10640000930B000013D54A01370910001309F9FF57
:106410001375F57F3379590193050C0093DAFA016E
:10642000630205109307F07F6302F51637048000BE
:1064300013193900336989001354DC0133642401D2
:1064400093153C00130515C09307000013972B000C
:106450003367F7001307F7FF9306E00033C95901CC
:10646000330AAA4063E0E61697A60100938686E108
:10647000131727003307D700032707003307D70078
:1064800067000700336BA400630E0B06630004046F
:1064900013050400EF109017930755FF1307C00171
:1064A000634CF702130BD001930485FF330BFB40C1
:1064B00033149400335B6901336B8B00B314990080
:1064C000130AD0C0330AAA406FF09FF3EF101014E4
:1064D000130505026FF05FFC130485FD331B890073
:1064E000930400006FF0DFFD336BA40063040B0224
:1064F00093040500130B0400130AF07F930B300084
:106500006FF05FF093040000130A0000930B10007B
:106510006FF05FEF93040000130AF07F930B2000ED
:106520006FF05FEE33648901630E040663000904B3
:1065300013050900EF10900D930755FF1307C001D5
:10654000634EF7021304D001930585FF3304F44032
:106550003319B90033548C0033642401B315BC00E3
:106560001307D0C03305A7406FF01FEE13050C00D2
:10657000EF10D009130505026FF01FFC130485FD11
:1065800033148C00930500006FF09FFD3364890184
:1065900063020402130409001305F07F930730001F
:1065A0006FF0DFEA93050000130500009307100069
:1065B0006FF0DFE9930500001305F07F93072000DB
:1065C0006FF0DFE86366640163128B4863E0B448F0
:1065D0009316FB0113D71400139CF401135B1B00EB
:1065E000B3E4E6001314840093DC8501B3EC8C0063
:1065F00093DA0C0193970C0193D70701139D850043
:1066000013050B0093850A002322F100EF1040755B
:1066100093050500930B050013950C011355050117
:10662000EF1040711304050093850A0013050B0059
:10663000EF1080771315050113D704013365A70008
:1066400093890B00637E8500330595019389FBFFD9
:1066500063689501637685009389EBFF33059501A7
:106660003304854093850A0013050400EF10406F42
:1066700093050500930B050013950C0113550501B7
:10668000EF10406B130B050093850A0013050400FF
:10669000EF108071939D04011315050193DD0D0129
:1066A000B3EDAD0013870B0063FE6D01B38D9D014B
:1066B0001387FBFF63E89D0163F66D011387EBFF12
:1066C000B38D9D0193960901B7040100B3E6E6007E
:1066D000B38D6D41138BF4FF33F76601337B6D018E
:1066E0001305070093050B0013D406012326D100E0
:1066F0002324E100EF1000642322A10093050B0086
:1067000013050400EF100063935B0D01930905006E
:1067100093850B0013050400EF10C061032781006F
:106720001304050013850B0093050700EF1080602C
:1067300003264100330535018326C10013570601A6
:106740003307A70063743701330494003705010051
:106750001305F5FF93540701B379A7009399090135
:106760003376A600B3848400B389C90063E89D0032
:106770001384060063949D0463723C05330CAC01E2
:106780003337AC0133079701B38DED001384F6FF67
:1067900063E6BC016394BC036362AC0363E69D00E3
:1067A000639EB401637C3C01330CAC013337AC0114
:1067B000330797011384E6FFB38DED00B3093C4125
:1067C000B3849D40B3373C01B384F4409305F0FF9C
:1067D00063889C1A93850A0013850400EF104058C3
:1067E000930505002324A10013950C011355050101
:1067F000EF1040542322A10093850A001385040062
:10680000EF10805A832681000327410013150501EC
:1068100093D7090133E5A700938D0600637EE50059
:1068200033059501938DF6FF636895016376E50066
:10683000938DE6FF33059501B304E54093850A0087
:1068400013850400EF10C051930505002322A10019
:1068500013950C0113550501EF10C04D130C0500E5
:1068600093850A0013850400EF10005493990901E1
:10687000032741001315050193D9090133E5A90048
:1068800093070700637E8501330595019307F7FFA2
:1068900063689501637685019307E7FF33059501EA
:1068A00093940D01B3E4F4009397040193D7070187
:1068B00093050B00B3098541138507002322F100DE
:1068C00093DD0401EF10004793050B00930A0500C8
:1068D00013850D00EF100046130C050093850D0085
:1068E00013850B00EF10004583274100130B0500B3
:1068F00013850B0093850700EF10C0433305850116
:1069000093D70A013385A70063768501B707010095
:10691000330BFB00B70601009386F6FF9357050182
:106920003377D50013170701B3FADA00B38767018D
:106930003307570163E8F900938504006390F90475
:106940006300070433853C019385F4FF636495037A
:106950006366F5006314F5026370ED0293161D0083
:1069600033BDA601B30C9D019385E4FF330595016A
:10697000138D06006314F5006304A70193E5150069
:106980001307FA3F6352E01293F775006380070222
:1069900093F7F50093064000638AD700938645007D
:1069A000B3B5B6003304B4009385060093177400A2
:1069B00063DA0700B70700FF9387F7FF3374F4002B
:1069C00013070A409307E07F63C2E71A9317D401C5
:1069D00093D53500B3E7B70013543400B706100061
:1069E0009386F6FF3374D400B70610801377F77FD1
:1069F0009386F6FF131747013374D4001319F90176
:106A00003364E400336724018320C1040324810438
:106A100083244104032901048329C103032A810338
:106A2000832A4103032B0103832BC102032C810220
:106A3000832C4102032D0102832DC1011385070020
:106A4000930507001301010567800000130AFAFF90
:106A5000130C00006FF01FB91389090013040B0019
:106A60009385040093870B00130720006380E710D1
:106A7000130730006382E70E13071000E392E7F07C
:106A800013040000930700006F00400913890A00F7
:106A90006FF09FFD37040800930500001309000004
:106AA000930730006FF05FFC93061000B386E6405A
:106AB00093078003E3C6D7FC9307F00163C4D706AE
:106AC000130AEA41B317440133D7D500339A45017D
:106AD000B3E7E700333A4001B3E747013354D4004A
:106AE00013F777006300070213F7F70093064000DF
:106AF000630AD70013874700B337F7003304F40065
:106B00009307070013178400634A07061317D4017D
:106B100093D73700B367F70013543400130700000E
:106B20006FF0DFEB930710FEB387E7401307000217
:106B3000B357F400130500006386E600130AEA4326
:106B400033154401336AB500333A4001B3E74701D6
:106B5000130400006FF0DFF837040800930700000B
:106B60001307F07F130900006FF05FE713040000C4
:106B7000930700001307F07F6FF05FE61304000037
:106B800093070000130710006FF05FE513D745016E
:106B9000B70710009387F7FF13D846019308050045
:106BA000930E05001377F77F1305F07F33F3B700DB
:106BB000130F0600B3F7D70093D5F5011378F87FCC
:106BC00093D6F601631AA700336E13011305E0FF95
:106BD000630C0E0867800000631AA80033E6C70044
:106BE0001305E0FF630A06086780000063100708CA
:106BF00033651301133515006316080033E6C7002B
:106C000063000606631A0500638ED50013051000A5
:106C10006396050067800000E39E06FE1305F0FF03
:106C200067800000E344E8FE635A07011305F0FFA4
:106C3000E38205FE1305100067800000E3E867FCAF
:106C4000631AF300E364DFFD13050000E3E0EEFFE9
:106C50006FF05FFCE36CF3FC13050000678000003D
:106C6000E31C05FE6FF09FFAE30AE8F61305000047
:106C7000E30608F86FF05FF9E31807F833651301CE
:106C8000133515006FF01FF813D74501B707100033
:106C90009387F7FF13D8460193080500930E05006C
:106CA0001377F77F1305F07F33F3B700130F060058
:106CB000B3F7D70093D5F5011378F87F93D6F60193
:106CC000631AA700336E130113052000630C0E082E
:106CD00067800000631AA80033E6C7001305200090
:106CE000630A060867800000631007083365130114
:106CF000133515006316080033E6C7006300060667
:106D0000631A0500638ED500130510006396050015
:106D100067800000E39E06FE1305F0FF6780000019
:106D2000E344E8FE635A07011305F0FFE38205FE22
:106D30001305100067800000E3E867FC631AF300A6
:106D4000E364DFFD13050000E3E0EEFF6FF05FFC9E
:106D5000E36CF3FC1305000067800000E31C05FEF4
:106D60006FF09FFAE30AE8F613050000E30608F85F
:106D70006FF05FF9E31807F8336513011335150059
:106D80006FF01FF8130101FA232C8104232631052B
:106D90003704100093D94501232A9104232061056B
:106DA000232E7103232C81031304F4FF232E1104DB
:106DB000232821052324410523225105232A910359
:106DC0002328A1032326B10393F9F97F9304050037
:106DD000930B0600138C06003374B40013DBF5012B
:106DE0006388090A9307F07F6386F91037098000EA
:106DF00013143400336424011359D5013369890015
:106E0000131D3500938919C0930C000013554C01D4
:106E1000370A1000130AFAFF1375F57F337A8A01D7
:106E200093840B00135CFC01630405109307F07F4F
:106E30006304F51637048000131A3A00336A8A0097
:106E400013D4DB013364440193943B00130515C054
:106E50009307000013972C003367F700B389A9004C
:106E60001307F7FF9306E000B34B8B01938A1900D9
:106E700063E0E61697960100938686441317270071
:106E80003307D700032707003307D7006700070041
:106E90003369A400630E09066300040413050400AB
:106EA000EF00D076930755FF1307C001634CF7023C
:106EB0001309D001130D85FF3309F9403314A401E0
:106EC00033D9240133698900339DA4019309D0C0CB
:106ED000B389A9406FF05FF3EF005073130505020B
:106EE0006FF05FFC130985FD33992401130D000039
:106EF0006FF0DFFD3369A40063040902130D050080
:106F0000130904009309F07F930C30006FF01FF019
:106F1000130D000093090000930C10006FF01FEF99
:106F2000130D00009309F07F930C20006FF01FEE0B
:106F300033647A01630E040663000A0413050A0031
:106F4000EF00D06C930755FF1307C001634EF702A3
:106F50001304D001930485FF3304F440331A9A00DC
:106F600033D48B0033644401B3949B009307D0C0A7
:106F70003385A7406FF0DFED13850B00EF0010693C
:106F8000130505026FF01FFC130485FD33948B007D
:106F9000930400006FF09FFD33647A0163020402E2
:106FA00013040A001305F07F930730006FF09FEA87
:106FB0009304000013050000930710006FF09FE991
:106FC000930400001305F07F930720006FF09FE803
:106FD00037070100130AF7FF135C0D0193DD04016D
:106FE000337D4D01B3F4440193050D001385040076
:106FF0002328E100EF001054930C05009385040052
:1070000013050C00EF0010532326A10093850D00FB
:1070100013050C00EF001052130B050093050D0033
:1070200013850D00EF0010518326C10093D70C018A
:107030003305D5003385A7006376D500032701010A
:10704000330BEB009356050133754501B3FC4C013E
:1070500013150501B3079501935C040133744401D2
:1070600093050D0013050400232AD1002326F10007
:10707000EF00504C2328A1009305040013050C00D9
:10708000EF00504B130A050093850C0013050C000C
:10709000EF00504A130C050093050D0013850C00FA
:1070A000EF005049032701013305450183264101C3
:1070B000935707013385A70063764501B7070100A1
:1070C000330CFC003706010093570501338C870110
:1070D0009307F6FF337AF5003377F700131A0A01A6
:1070E000135D0901330AEA003379F9003387460159
:1070F00093050900138504002328E100232EC10015
:10710000EF00504393850400232CA10013050D00CC
:10711000EF005042232AA10093050D0013850D00B6
:10712000EF005041930405009305090013850D00FD
:10713000EF00504083264101032781013305D5002C
:10714000935707013385A7006376D5000326C10155
:10715000B384C400B70601009387F6FF935D050171
:10716000B3849D00B37DF5003377F70093050900E4
:1071700013050400939D0D01B38DED00232CD10068
:10718000EF00503B93050400232AA10013050D00D6
:10719000EF00503A93050D001304050013850C0011
:1071A000EF005039130D05009305090013850C00FD
:1071B000EF0050380327410133058500935707013D
:1071C0003385A7006376850083268101330DDD00BA
:1071D00083270101B70601009386F6FF330BFB00FE
:1071E000B377D5003377D70093970701B387E700CC
:1071F000333A4B01B387870133844701330BBB011B
:1072000033079400B33DBB01B306B70133BC87011C
:1072100033344401935705013337970033648C00AE
:10722000B3BDB6013304F400B36DB7013304B40148
:107230003304A40193D77601131494003364F4004B
:107240008327C10093149B00135B7B01B3E4F4001C
:10725000B334900093979600B3E46401B3E4F40070
:107260009317740063D2071293D7140093F4140099
:10727000B3E497009317F401B3E4F400135414003B
:107280001387FA3F6356E01093F774006380070298
:1072900093F7F40093064000638AD7009387440075
:1072A000B3B49700330494009384070093177400D9
:1072B00063DA0700B70700FF9387F7FF3374F40022
:1072C00013870A409307E07F63C6E71893DA340018
:1072D0009314D401B3E4540113543400B7071000DD
:1072E0009387F7FF3374F4009377F77F37071080A5
:1072F0001307F7FF939747013374E400939BFB0157
:107300003364F400B36774018320C105032481054D
:107310001385040003290105832441058329C10441
:10732000032A8104832A4104032B0104832BC10314
:10733000032C8103832C4103032D0103832DC10200
:10734000938507001301010667800000930B0B0073
:107350001304090093040D0093870C001307200009
:10736000638AE70E13073000638CE70C13071000E5
:10737000E398E7F013040000930400006F00800816
:10738000930B0C006FF09FFD938A09006FF05FEF85
:1073900093061000B386E64093078003E3CCD7FC46
:1073A0009307F00163C4D706938AEA41B3175401E7
:1073B00033D7D400B3945401B3E7E700B33490005B
:1073C000B3E497003354D40093F77400638007024A
:1073D00093F7F40013074000638AE70093874400A3
:1073E000B3B4970033049400938407009317840088
:1073F00063CA07069317D40193D43400B3E497000B
:1074000013543400130700006FF05FED930710FE74
:10741000B387E74013060002B357F40013070000D8
:107420006386C600938AEA4333175401B364970016
:10743000B3349000B3E49700130400006FF0DFF85A
:1074400037040800930400001307F07F930B00003B
:107450006FF0DFE813040000930400001307F07FCF
:107460006FF0DFE71304000093040000130710001F
:107470006FF0DFE6370810001308F8FF130101FE74
:10748000B378B80013D745019357D5013378D800A6
:10749000232821011379F77F13973800B3E7E7001A
:1074A00093D8F60113D74601131838009356D60126
:1074B000232A910033E30601232E1100232C81009F
:1074C000232631011377F77F9306F07F93D4F501DC
:1074D00013153500131636006316D700B366C300C4
:1074E0006394060093C818003308E9406394983AFF
:1074F0006354001F631207143367C3006314070C3F
:107500009306F07F13070800631CD830B3E6A7008A
:1075100063980630930700001305000093968700D8
:1075200063DE0600130717009306F07F630CD77421
:10753000B70680FF9386F6FFB3F7D7009396D7017F
:107540001355350033E5A6009306F07F93D7370037
:10755000631ED7003365F50093070000630805003C
:10756000B70708001305000093040000B7061000D9
:107570009386F6FFB3F7D700B70610801377F77F2F
:107580009386F6FF13174701B3F7D700B3E7E70079
:10759000370700801347F7FF8320C10103248101CF
:1075A0009395F401B3F7E70033E7B7008324410173
:1075B000032901018329C10093050700130101027A
:1075C000678000009305F8FF639C05043306C5003F
:1075D0003335A600B3876700B387A70013071000F1
:1075E000130506009396870063DC06221307170035
:1075F0009306F07FE300D7F2B70680FF9386F6FF8D
:10760000B3F6D70093551500137515009397F6013F
:1076100033E5A50033E5A70093D716006F0040209F
:107620001307F07F6314E80233E7A70063000762E3
:107630001307F07F6F00C01E1307F07FE306E9FE1B
:10764000370780003363E3009305080013078003C6
:10765000634EB7061307F0016342B7041307000235
:107660003307B740B356B6003318E3003316E600CD
:107670003368D8003336C0003368C800B355B30050
:107680003308A800B385F500B337A800B387F50029
:1076900013050800130709006FF0DFF41307000259
:1076A0003358B300930600006388E5009306000496
:1076B000B385B640B316B30033E6C6003336C00018
:1076C0003368C800930500006FF09FFB3368C30068
:1076D000333800016FF01FFF630A080E631E0908AC
:1076E000B3E6A700639206029307F07F6318F700E2
:1076F0003365C30093070000E30205E2930703002C
:10770000130506006F00C0119306F0FF631CD8003C
:107710003305C500B38767003336C500B387C7009C
:107720006FF05FEC9306F07F1348F8FFE302D7FC9D
:107730009306800363C606099306F00163CA060533
:1077400093050002B3850541B3580501B396B70010
:107750003315B500B3E616013335A00033E5A600B6
:1077600033D807013305C50033086800B337C500B7
:10777000B307F8006FF01FE79306F07FE30AD7F630
:10778000B706800033080041B3E7D7006FF05FFA17
:1077900093080002B3D6070193050000630818019F
:1077A0009305000433880541B395070133E5A5002F
:1077B0003335A00033E5A600130800006FF09FFAF0
:1077C00033E5A7003335A0006FF01FFF1307190042
:1077D0009375F77F9306100063C8B60833E7A700D8
:1077E0006314090663080744B366C3001307000067
:1077F000638806023306C5003335A600B3876700E9
:10780000B387A700939687001305060063DA060086
:10781000370780FF1307F7FFB3F7E70013071000E0
:1078200093767500E38C06CE9376F5001306400040
:10783000E386C6CE9306450033B5A600B387A700FE
:10784000138506006FF09FCD630C073E3368C300BD
:10785000E30008DEB7074000130500001307F07FC0
:10786000930400006FF09FCB9306F07FE304D7CA28
:107870003306C50033886700B337A6003308F80025
:107880001315F801135616003365C50093571800F9
:107890006FF01FF9635E000F6312070A3367C300BE
:1078A000E30007C69306F8FF639E06023306C54051
:1078B0003335C500B3876740B387A740130710006F
:1078C0001305060093968700E3DC06F43704800076
:1078D0001304F4FF33F4870093090500130907002C
:1078E0006F0000271307F07FE300E8D4130780033D
:1078F000634AD7081307F001634ED7041307000249
:107900003307D740B355D6003318E3003316E600EB
:107910003368B8003336C0003368C800B356D300AC
:1079200033080541B386D740B3370501B387F64026
:1079300013050800130709006FF0DFF81307F07F45
:10794000E304E9CE370780003363E30093060800C1
:107950006FF0DFF9130700023358D300130400005F
:107960006388E60013040004B306D4403314D30044
:107970003366C4003336C0003368C8009306000085
:107980006FF01FFA3368C300333800016FF01FFF38
:10799000630A080E631E0908B3E6A7006390060297
:1079A0009307F07F6316F7003365C3006308052A69
:1079B00093070300130506006F00C00F9306F0FF46
:1079C000631ED8003305A640B307F3403336A60044
:1079D000B387C740938408006FF0DFEE9306F07F13
:1079E0001348F8FFE302D7FC9306800363C6060939
:1079F0009306F00163CA060593050002B3850541AD
:107A0000335E0501B396B7003315B500B3E6C60182
:107A10003335A00033E5A60033D807013305A6406F
:107A200033080341B337A600B307F8406FF09FFA5D
:107A30009306F07FE30AD7F6B706800033080041CB
:107A4000B3E7D7006FF05FFA130E0002B3D6070159
:107A5000930500006308C8019305000433880541BD
:107A6000B395070133E5A5003335A00033E5A60043
:107A7000130800006FF09FFA33E5A7003335A0002C
:107A80006FF01FFF130719001377F77F930610009D
:107A900063CAE608B3E6A7003367C30063140906A8
:107AA000639E06006302071C93070300130506008C
:107AB00013070000938408006FF09FD6630007044B
:107AC000B306C540B335D500338767403307B740A9
:107AD0009315870063DC05003305A640B307F34028
:107AE0003336A600B387C7406FF09FFC33E5E6004E
:107AF000630A050C930707001385060013070000AF
:107B00006FF01FD2639C06006308071693070300FB
:107B100013050600938408006FF09FB1E30A07B0D5
:107B20006FF05FD3B309C540338467403338350104
:107B3000330404411317840063520708B309A640B5
:107B40003304F340B33736013304F4409384080020
:107B5000630E040613050400EF00402B130785FF96
:107B60009307F00163CCE70693070002B387E74071
:107B70003314E400B3D7F90033E487003395E90008
:107B80006340270B33072741930717009306F00143
:107B900063CEF604130700023307F7403356F500AF
:107BA000B316E4003315E500B3E6C6003335A00094
:107BB00033E5A600B357F4006FF05FF433E58900B6
:107BC000E31805F8930700006F00800A1385090089
:107BD000EF00C023130505026FF05FF8130485FD65
:107BE00033948900130500006FF09FF9130717FE07
:107BF000130600023357E400930600006388C700B1
:107C000093060004B386F640B316D4003365D5005E
:107C10003335A0003365A700930700006FF01FEE17
:107C2000B70780FF9387F7FF3307E940B377F40086
:107C30006FF01FBF93070300130506006FF01FECE2
:107C400093070300130506006FF09F9E9307000043
:107C5000130500001307F07F6FF05F8C930700009F
:107C6000938408006FF09F8B9307000013050000BA
:107C7000130700006FF0DFBE13050000B7074000D8
:107C80006FF0DFBD93070000130500006FF01F8B3E
:107C9000130101FF2326110023248100630405083A
:107CA00013040500EF0080161307E0419307A000BE
:107CB0003307A74063C0A7069307B000B387A74068
:107CC00013055501B357F4003314A4003705100011
:107CD0001305F5FFB7061080B3F7A7001377F77FFA
:107CE0009386F6FF13174701B3F7D700B3E7E70012
:107CF000130504008320C10003248100370700809E
:107D00001347F7FF33F7E70093050700130101015D
:107D100067800000130555FFB317A400130400008B
:107D20006FF0DFFA93070000130400001307000050
:107D30006FF0DFF9130605001305000093F6150038
:107D4000638406003305C50093D51500131616008D
:107D5000E39605FE678000006340050663C60506DE
:107D600013860500930505001305F0FF630C06025A
:107D700093061000637AB6006358C000131616000D
:107D800093961600E36AB6FE1305000063E6C5008D
:107D9000B385C5403365D50093D61600135616003B
:107DA000E39606FE6780000093820000EFF05FFB21
:107DB00013850500678002003305A04063D80500E5
:107DC000B305B0406FF0DFF9B305B0409382000017
:107DD000EFF01FF93305A040678002009382000096
:107DE00063CA0500634C0500EFF09FF7138505009B
:107DF00067800200B305B040E35805FE3305A0409C
:107E0000EFF01FF63305B04067800200B7070100AE
:107E1000637AF5029307F00FB3B7A7009397370083
:107E2000130700023307F740B357F5001785010029
:107E30001305C54CB307F50003C507003305A7407C
:107E4000678000003707000193070001E36AE5FC43
:087E5000930780016FF0DFFCD5
:02000004800278
:1000000049444C4500000000482FFEFF102FFEFF22
:100010001E2FFEFF2C2FFEFF342FFEFF5830FEFF59
:100020002030FEFF2E30FEFF3C30FEFF4430FEFF4E
:10003000546D722053766300DC35FEFFDC35FEFF25
:10004000DC35FEFF5A36FEFF2A36FEFF5036FEFF35
:10005000DC35FEFFDC35FEFF5A36FEFF2A36FEFF9A
:10006000546D725100000000286E756C6C29000000
:10007000DE43FEFFDC45FEFFD245FEFFDC45FEFF12
:10008000DC45FEFFDC45FEFFDC45FEFF5C44FEFF79
:10009000DC45FEFFDC45FEFF1444FEFF6A44FEFF24
:1000A000DC45FEFF1E44FEFF2844FEFF2844FEFF01
:1000B0002844FEFF2844FEFF2844FEFF2844FEFF9C
:1000C0002844FEFF2844FEFF2844FEFFDC45FEFFD7
:1000D000DC45FEFFDC45FEFFDC45FEFFDC45FEFFA8
:1000E000DC45FEFFDC45FEFFDC45FEFFDC45FEFF98
:1000F000DC45FEFFDC45FEFFDC45FEFFDC45FEFF88
:10010000DC45FEFFDC45FEFFDC45FEFFDC45FEFF77
:10011000DC45FEFFDC45FEFFDC45FEFFDC45FEFF67
:10012000DC45FEFFDC45FEFFDC45FEFFDC45FEFF57
:10013000DC45FEFFDC45FEFFDC45FEFFDC45FEFF47
:10014000DC45FEFFDC45FEFFDC45FEFFDC45FEFF37
:10015000DC45FEFFDC45FEFFDC45FEFFDC45FEFF27
:10016000DC45FEFFDC45FEFFDC45FEFFDC45FEFF17
:100170008E44FEFF3A45FEFFDC45FEFFDC45FEFFF8
:10018000DC45FEFFDC45FEFFDC45FEFFDC45FEFFF7
:10019000DC45FEFF8644FEFFDC45FEFFDC45FEFF3E
:1001A0008E45FEFF9445FEFFDC45FEFFDC45FEFF6D
:1001B000A244FEFFDC45FEFF8845FEFFDC45FEFF56
:1001C000DC45FEFFAC45FEFF6D69616F750A0000FE
:1001D0006D69616F75320A0068756E6772790A0021
:1001E0004572726F7220696E20666C6F7073207436
:1001F00061736B73200D0A00436865636B54696D0E
:1002000065720000000000004D617468310000005C
:100210004D617468320000004D6174683300000065
:100220004D617468340000006AE67F50274C41C17C
:100230005305A3923ADD5E4082E2C7985B53A24029
:10024000B29DEFA7C6B18CC0FCA9F1D24D62503F60
:10025000AE47E17A145678C0CDCCCCCC8CBCDF4014
:1002600039D6C56D340000C0000000000000164003
:10027000FCA9F1D24D6250BFE5D022DBF93E284007
:10028000EC68FEFF0068FEFF0C68FEFF0068FEFFE2
:10029000D868FEFF0068FEFF0C68FEFFEC68FEFFFA
:1002A000EC68FEFFD868FEFF0C68FEFFD867FEFF13
:1002B000D867FEFFD867FEFF1468FEFFA070FEFF40
:1002C000A070FEFFC470FEFF9470FEFF9470FEFFEE
:1002D0008471FEFFC470FEFF9470FEFF8471FEFF08
:1002E0009470FEFFC470FEFF9070FEFF9070FEFFE2
:1002F0009070FEFF8471FEFF0001020203030303FE
:1003000004040404040404040505050505050505A5
:100310000505050505050505060606060606060685
:10032000060606060606060606060606060606066D
:100330000606060606060606070707070707070755
:10034000070707070707070707070707070707073D
:10035000070707070707070707070707070707072D
:10036000070707070707070707070707070707071D
:100370000707070707070707080808080808080805
:1003800008080808080808080808080808080808ED
:1003900008080808080808080808080808080808DD
:1003A00008080808080808080808080808080808CD
:1003B00008080808080808080808080808080808BD
:1003C00008080808080808080808080808080808AD
:1003D000080808080808080808080808080808089D
:1003E000080808080808080808080808080808088D
:0803F0000808080808080808C5
:1003F8001000000000000000017A5200017C010199
:100408001B0D02004C00000018000000844CFEFF89
:10041800DC05000000440E307089039507810188CF
:100428000292049305940696089709980A990B9ADC
:100438000C0370020AC144C844C944D244D344D40A
:1004480044D544D644D744D844D944DA440E004469
:100458000B00000050000000680000001052FEFF72
:100468000005000000440E50748802890393059922
:100478000B810192049406950796089709980A9AA1
:100488000C9B0D0320010AC144C844C944D244D37B
:1004980044D444D544D644D744D844D944DA44DB78
:0804A800440E00440B000000AB
:1004BC00AAAAAAAA08000000FC8F010004000000F0
:040000058000004037
:00000001FF
